:02000004100DDD
:1000000000C00208334B0D100D000000A14B0D1075
:1000100000000000000000000000000000000000E0
:100020000000000000000000000000009D4B0D10CB
:1000300000000000000000009D4B0D109D4B0D10B6
:100040009D4B0D109D4B0D109D4B0D109D4B0D109C
:100050009D4B0D109D4B0D109D4B0D109D4B0D108C
:100060009D4B0D109D4B0D109D4B0D109D4B0D107C
:100070009D4B0D109D4B0D109D4B0D109D4B0D106C
:100080009D4B0D109D4B0D109D4B0D109D4B0D105C
:100090009D4B0D109D4B0D109D4B0D109D4B0D104C
:1000A0009D4B0D109D4B0D109D4B0D109D4B0D103C
:1000B0009D4B0D109D4B0D109D4B0D109D4B0D102C
:1000C00010B5064C2378002B07D1054B002B02D02E
:1000D000044800E000BF0123237010BDECA7020814
:1000E00000000000508C0D10044B10B5002B03D005
:1000F0000349044800E000BF10BDC04600000000F6
:10010000F0A70208508C0D100021124B124A10B5B6
:10011000D8601C68002C06DB914202D101204042CD
:1001200010BD0131F5E79142F8D00121996000211D
:100130001C69002C03DA9142F0D00131F8E79142BA
:10014000ECD0A0220368120600209342E8D01800E9
:10015000E6E7C04600002340983A00001FB50023A0
:100160000193D82300049B05C018029001AB02A89C
:100170000C000393FFF7C8FF002801D1019B236007
:1001800004B010BD13B5084BC47A986801A9C0B279
:10019000FFF7E4FF002803D1019B9C42804116BD7C
:1001A00001204042FBE7C046E8AD02081FB5064B00
:1001B0000004C018029001AB02A801910393FFF75D
:1001C000A3FF05B000BDC0460001003610B5034BCB
:1001D000C17A9868C0B2FFF7E9FF10BDE8AD020828
:1001E000F0B50F000400002685B0BE4201D100200A
:1001F0003EE0A0221F4BD2009A582378032A04D055
:10020000092B02D801361034EFE71B4A0A33DB0012
:1002100099580029F6D0D3185B6801AD2B7163782B
:1002200001916B71A3782900AB71E378A068EB7141
:1002300023792B7263796B72E3886B8102F0B0FBD8
:10024000002815D1237B2900AB71637BA068EB717B
:10025000E3896B8102F04AFB002809D1A06802F013
:1002600025FC002804D1A06802F008FC0028C9D0B1
:1002700005B0F0BD00002140E8AD020870B50600F1
:100280000024104AA3019B180F491A68A3015B18A8
:100290001B68002A04DA0134102CF2D1002070BD52
:1002A000002BF8DB094B3100E518AD01280002F006
:1002B0001DFB0028F3D1280002F0E0FB0028EAD063
:1002C000EDE7C04604202440242024408090000113
:1002D00073B50E0004000025B54201D1002076BDA3
:1002E0006A462378694613706378E0685370A37890
:1002F0009370E378D370A388938002F06BFE00289C
:10030000EDD16A46A37969461370E379E0685370CA
:10031000237A93706389938002F000FE0028DED177
:10032000E06802F0CDFE0028D9D1E06802F0AEFE10
:1003300010340028D3D10135CEE773B50E00040088
:100340000025B54201D1002076BD6A462378694672
:1003500013706378E0685370A3789370E378D37078
:10036000A388938002F036FD0028EDD16A46A37978
:1003700069461370E379E0685370237A9370638958
:10038000938002F0CBFC0028DED1E06802F0A2FDF1
:100390000028D9D1E06802F079FD10340028D3D1CB
:1003A0000135CEE7F0B50F000400002685B0BE424F
:1003B00002D1002005B0F0BD236801AD019323797F
:1003C00029002B71637960696B71A379AB71E37953
:1003D000EB71237A2B72637A6B7263896B8102F003
:1003E000DDFB0028E6D1237B2900AB71637B6069CC
:1003F000EB71A37B2B72238A6B8102F06FFB0028C9
:10040000D8D1606902F066FC0028D3D1606902F09F
:100410003DFC18340028CDD10136C8E730B5174B64
:1004200085B001930D2301AD2B71437804006B71EE
:1004300083782900AB71C378EB7103792B72437910
:100440006B72C38880686B8102F0AAFA002813D10E
:10045000237B2900AB71637BA068EB71E3896B811F
:1004600002F044FA002807D1A06802F01FFB002820
:1004700002D1A06802F002FB05B030BD00C0020846
:10048000B02310B55B055B78124C232B1BD00B21DE
:100490002000FFF7A5FE00281AD10F48FFF7EEFE57
:1004A000002815D10A210D48FFF712FF00280FD1AF
:1004B00004210B48FFF741FF002809D10121094819
:1004C000FFF770FF04E02000FFF7A8FF0028DED050
:1004D00010BDC0462C7C0D10287B0D10347B0D10F8
:1004E000D47B0D10147C0D1010B501210148FFF7CD
:1004F00077FE10BDDC7C0D100022124B124910B5A6
:10050000D8601C68002C05DB8A4201D1012010BD97
:100510000132F6E78A42F9D001229A6000220B49A3
:100520001C69002C03DA8A42F0D00132F8E78A42D3
:10053000ECD0A0220368120600209342E7D01800F6
:10054000E5E7C04600002340983A00000094357764
:1005500010B5D42488B005930A9BA40506930B9B81
:100560000094029002AC68460194039104920793B0
:10057000FFF7C2FF08B010BD00B5064B89B000936D
:10058000029002AB6846019303910492FFF7B4FF17
:1005900009B000BD000B003510B5074C88B00094C1
:1005A000029002AC68460194039104920593FFF710
:1005B000A3FF08B010BDC046000E003500B5064BC5
:1005C00089B00093029002AB6846019303910492B4
:1005D000FFF792FF09B000BD000C003510B588B0E0
:1005E00005930A9B074C06930B9B0094029002AC68
:1005F00068460194039104920793FFF77DFF08B0CA
:1006000010BDC046000D003500B5054B89B0009304
:10061000029002AB68460193FFF76EFF09B000BD80
:10062000000A003500B5054B89B00093029002AB7B
:1006300068460193FFF760FF09B000BD0005003573
:1006400000B5064B89B00093029002AB6846019357
:1006500003910492FFF750FF09B000BD000400357C
:100660001FB5054B02900093684602AB01930391BE
:10067000FFF742FF05B000BD001000357FB5064B07
:100680000390019301A803AB029304910592FFF735
:1006900033FF07B000BDC0460011003510B5074C50
:1006A00086B00094029002AC6846019403910492D3
:1006B0000593FFF721FF06B010BDC04600120035BC
:1006C00010B5074C86B00094029002AC68460194C5
:1006D000039104920593FFF70FFF06B010BDC046CB
:1006E000000900357FB5054B0390019301A803ABCA
:1006F0000293FFF701FF07B000BDC04600060035BA
:100700007FB5064B0390019301A803AB02930491BC
:100710000592FFF7F1FE07B000BDC04600070035A7
:100720007FB5054B0390019301A803AB029304919D
:10073000FFF7E2FE07B000BD000800357FB5064BAD
:100740000390019301A803AB029304910592FFF774
:10075000D3FE07B000BDC0460002003510B5074CFF
:1007600086B00094029002AC684601940391049212
:100770000593FFF7C1FE06B010BDC046000100356D
:1007800010B58CB006930E9B0A4C07930F9B0194F7
:100790000893109B03900993119B03AC0A93129B3F
:1007A00001A80294049105920B93FFF7A5FE0CB0EB
:1007B00010BDC04600030035F0B58DB01D0012AB72
:1007C00040CB02921B780F000393002305AA04A9D3
:1007D0000493059300F03DF9041E3BD1204B3A00F1
:1007E00000930599029B049806F08EFC002834DDE6
:1007F000022007AA06A9FF300694079401F0AEF97B
:10080000002803D12900069800F0F4FF812007AAF0
:1008100006A9400001F0A2F9652400281ED131008C
:10082000069800F077FD041E14D108A9380000F0E6
:1008300028F9041E0ED131000B9800F063FB041E52
:1008400008D1039A29000B9800F03AF9040008989F
:1008500006F0F0FB20000DB0F0BD14246442F9E76F
:10086000005F2D00F0B51F00002387B002910392B6
:1008700004A905AA0493059300F0EBF8041E2ED1F9
:10088000059800F07FF8040006F0FEFE051E31D04A
:100890001A4B0200009305992300049806F034FCDB
:1008A000002822DD280006F01FFC061E20D00100D3
:1008B000134800F09FF8002814D00069002811D0D8
:1008C000039B220000930197029B2900FFF774FF0E
:1008D0000400300006F0AEFB280006F0DFFE20002A
:1008E00007B0F0BD01246442F3E714246442F3E747
:1008F0000524FBE764246442F1E7C046005F2D0055
:10090000EC7C0D1010B5010004000B4806F0CAFF86
:10091000002398420DD02100084806F0C3FF0123B0
:10092000002806D02100064806F0BCFF43424341A0
:100930005B00180010BDC046F37D0D10FC7D0D104E
:10094000087E0D1010B5010004000B4806F0AAFF48
:10095000002398420DD02100084806F0A3FF012390
:10096000002806D02100064806F09CFF4342434180
:100970005B00180010BDC0460D7E0D10167E0D10D8
:100980001E7E0D100323584380089843043070479F
:10099000F8B5C3680D000860062B21D18468124F9A
:1009A000002C01D12000F8BD266A002E06D03100AF
:1009B0000E4806F077FF002802D16C602468EFE74C
:1009C00031000B4806F06EFF002801D1AC60F5E75E
:1009D0003100380006F066FF0028EFD1EC60EDE74B
:1009E00002204042DFE7C046357E0D10267E0D1006
:1009F0002C7E0D10F0B507000D00002491B001AE63
:100A0000002D02D1280011B0F0BD296A002904D0C0
:100A1000380006F047FF0028F4D0AB68002B06D062
:100A20000E2C12D8A200955101341D00E8E72B6866
:100A3000002BFAD1002C0AD0013CA3009B591B6863
:100A4000002BF2D1002CF7D1EFE70025DAE72500E3
:100A5000D8E7F8B50E002E21170006F015FF041E8A
:100A60000CD0451C2E21280006F00EFF002805D0D2
:100A7000001B0138386000203560F8BD1620404268
:100A8000FBE770B5050000200C0006F0B9FA28005D
:100A900006F02AFB002803D02100FFF779FF70BD84
:100AA00005204042FBE7002304220133002901D145
:100AB000904203D952001D2BF7D102331800704722
:100AC000F0B589B005900C000100C24807920027DC
:100AD000FFF790FFB84200D145E18568069702957F
:100AE0000497029B002B00D08AE0EB68062B00D015
:100AF00039E12E00B84F31003800FFF77BFF079A2D
:100B0000037E9A4200D0DEE03100B448FFF772FF66
:100B10008369237029003800FFF76CFF2278037E79
:100B20009A4200D1A8E12D68002DF3D12900AC48EC
:100B3000FFF760FF002806D02300FF335B7B012B0B
:100B400001D18369A3602900A648FFF753FF00285D
:100B500008D02300FF339B7A012B03D1C3685A1EB0
:100B6000934163702900A048FFF744FF002808D094
:100B70002300FF331B7B012B03D1C3685A1E934113
:100B8000E37029009948FFF735FF002806D02300BD
:100B9000FF331B7B012B01D183692371290094480A
:100BA000FFF728FF002809D02300FF331B7E012B0D
:100BB00004D1C3685A1E9341E21CD37729008D48A3
:100BC000FFF718FF002800D1A6E0C368052B00D06E
:100BD000A2E082682300200012331530FF33FF307B
:100BE000002A00D198E01978012903D119009669EB
:100BF000F5390E700133984200D18DE01268EFE7AD
:100C000002997D48FFF7F6FE002804D0836801931F
:100C1000019B002B03D1029B1B68029361E70199A2
:100C20007648FFF7E7FE00284AD0036974491800A8
:100C3000039306F037FE002842D07249039806F06D
:100C400031FE00283CD000266F4AB3009958039823
:100C500006F028FE071E05D00136172EF4D1052711
:100C6000183E7F4201996948FFF7C4FE002801D071
:100C70008369069301996648FFF7BCFE002804D0FB
:100C8000C1698069FFF70FFF0490731C18D0049BA3
:100C9000002B15DD92227300E31852009A5C012AA2
:100CA00004D1320006990A32D20011512622FF32B5
:100CB0009B5C012B04D10A36F600049BA6197360D5
:100CC000019B1B68A3E73668002E00D012E721E7DE
:100CD0004C49380006F0E6FD002800D0FFE0310066
:100CE0004A48FFF787FE002806D02300FF331B7C0D
:100CF000012B01D18369636131004548FFF77AFE1A
:100D0000002800D1EBE02300FF331B7C012B00D037
:100D1000E5E08369A361E2E029003E48FFF76AFE4F
:100D2000002817D0C368052B14D182682300200047
:100D300015331830FF33FF30002A0BD01978012902
:100D400003D119009669F5390E700133984201D02C
:100D50001268F1E729003048FFF74CFE002835D033
:100D600000278369A37005992C48FFF743FE0028EC
:100D700058D000258668002E54D031002448FFF753
:100D800039FE00280BD063191A001A32FF3212788C
:100D9000012A04D102326A439B1882699A623100A7
:100DA0001F48FFF727FE00280BD063191A001932DD
:100DB000FF321278012A04D102326A439B188269F9
:100DC0005A6202350A2D2DD03668D4E7A07007008C
:100DD000C9E7C046F37D0D105C7D0D10117D0D102F
:100DE000187D0D103A7E0D10227D0D102A7D0D10FC
:100DF000397D0D10407D0D10F57C0D10427E0D10DB
:100E0000FF7C0D10047D0D10C0A00208927E0D1015
:100E10000C7D0D104A7D0D10577D0D105F7D0D105E
:100E2000697D0D1005992F48FFF7E4FD051E20D0C0
:100E300001002D48FFF7DEFD00280AD02423FF33F0
:100E4000E35C012B05D1C3685A1E934122004D3249
:100E5000137029002548FFF7CDFD002809D0912304
:100E60005B00E35C012B04D1C3684C345A1E9341F0
:100E70002370380009B0F0BD29001D48FFF7BAFD06
:100E8000002800D152E68668002E00D14EE63100DF
:100E90001848FFF7AFFD002821D007691649380030
:100EA00006F000FD002800D012E731001348FFF7DC
:100EB000A1FD002806D02300FF339B7B012B01D12D
:100EC0008369E36031000E48FFF794FD002806D0E7
:100ED0002300FF33DB7B012B01D18369236136685B
:100EE000D2E7C0466F7D0D107B7D0D10877D0D1004
:100EF000F57C0D10427E0D10FF7C0D10927E0D10C2
:100F00000C7D0D10F8B507000C000100BA48FFF782
:100F100071FDBA4E051E2AD001003000FFF76AFDB0
:100F2000002808D0230068331B78012B03D1006907
:100F3000FFF708FD20702900B148FFF75BFD00288E
:100F400008D0230069331B78012B03D10069FFF718
:100F5000D9FC60702900AB48FFF74CFD002806D093
:100F600023006A331B78012B01D18369A3703900F8
:100F7000A548FFF73FFD051E2AD001003000FFF70E
:100F800039FD002808D023006B331B78012B03D1D7
:100F90000069FFF7D7FCE07029009948FFF72AFDA8
:100FA000002808D023006C331B78012B03D1006983
:100FB000FFF7A8FC207129009248FFF71BFD0028CD
:100FC00006D023006D331B78012B01D18369637137
:100FD00039008E48FFF70EFD051E00D184E00100A8
:100FE0003000FFF707FD002808D023006E331B7880
:100FF000012B03D10069FFF7A5FCA07129008048EF
:10100000FFF7F8FC002808D023006F331B78012B72
:1010100003D10069FFF776FCE07129007948FFF7FA
:10102000E9FC002806D0230070331B78012B01D186
:101030008369237229007648FFF7DCFC002808D07A
:10104000230071331B78012B03D1C3685A1E9341CF
:10105000637229006F48FFF7CDFC002808D02300F9
:1010600072331B78012B03D1C3685A1E9341A372BC
:1010700029006948FFF7BEFC002808D0230073331D
:101080001B78012B03D1C3685A1E9341E3722900D8
:101090006248FFF7AFFC002808D0230074331B78A8
:1010A000012B03D1C3685A1E9341237329005C4866
:1010B000FFF7A0FC002808D0230075331B78012B14
:1010C00003D1C3685A1E9341637329005548FFF743
:1010D00091FC002808D0230076331B78012B03D124
:1010E000C3685A1E9341A37339004F48FFF782FC2F
:1010F000050001003000FFF77DFC002808D0230028
:1011000077331B78012B03D10069FFF71BFC207498
:1011100029003C48FFF76EFC002808D023008C33E0
:101120001B78012B03D12300826964331A702900D4
:101130003E48FFF75FFC00282AD000268768002F72
:1011400026D039003A48FFF755FC00280AD0A319E9
:101150001A0078321278012A04D1023272439B18A5
:1011600082695A6139003348FFF744FC00280AD0ED
:10117000A3191A0079321278012A04D1023272437B
:101180009B1882699A6102360A2E01D03F68D6E721
:1011900029002948FFF72EFC00282BD00025032723
:1011A0008668002E26D031002148FFF723FC002856
:1011B0000AD063191A0082321278012A04D13A0047
:1011C0006A439B188269DA6331001A48FFF712FC00
:1011D00000280AD063191A0083321278012A04D138
:1011E0003A006A439B1882691A6402350A2D01D0BD
:1011F0003668D6E70020F8BD997D0D109D7D0D1055
:10120000A87D0D10B07D0D10B47D0D10B77D0D10B3
:10121000BE7D0D10C67D0D10E57D0D10A37E0D1059
:10122000AD7E0D10B47E0D10CB7D0D10CF7D0D1059
:10123000697D0D100C7D0D10DD7D0D1070B5040065
:101240000D0086B00021142201A806F05BFA2900E7
:101250002000FFF7CFFB0400002C18D021001C4811
:10126000FFF7C8FB0028F7D00569002D0AD0194EFA
:101270002900300006F016FB00280BD1310001A830
:1012800006F01AFB210001A8FFF7B4FB04002000C0
:1012900006B070BD104E2900300006F003FB002898
:1012A000ECD029000D4806F0FDFA0028E6D00C4EDF
:1012B0002900300006F0F6FA0028DFD0290009489E
:1012C00006F0F0FA0028DDD121000748C1E7C0464A
:1012D000427E0D106A7E0D10537E0D105A7E0D1049
:1012E000627E0D10477E0D104D7E0D1010B5FFF77C
:1012F00081FB0124002809D08168002906D0044818
:10130000FFF778FB002801D0C468E4B2200010BDCC
:10131000EB7D0D10F0B5050085B000200C0005F048
:101320006FFE280005F0E0FE0190002800D14BE29E
:101330000100A148FFF75EFB051E00D0B4E00123C9
:101340005B42009301999D48FFF754FB051E00D0B6
:10135000EEE001235B42009301999948FFF74AFBB5
:10136000051E00D03EE101235B42009301999548A0
:10137000FFF740FB071E00D122E2934E0100300030
:10138000FFF75CFF390005003000FFF7AFFF0600F4
:10139000002D00D1F6E12869FFF7D4FA2300773356
:1013A00020741E70894E39003000FFF747FF390066
:1013B00005003000FFF79AFF002D00D1E6E1230081
:1013C000AA6964331A702833187039008048FFF70F
:1013D00011FB051E00D1E6E101007E48FFF72EFF5C
:1013E000290006007B48FFF781FF0390002E00D103
:1013F000D0E1B369029329007748FFF71FFF290066
:1014000006007548FFF772FF002E00D1C7E1B669EC
:10141000230022002100143378323C31029D5E60AB
:101420001D606D462D7B0833507015700232994255
:10143000F4D139006948FFF7DDFA061E00D1BFE19B
:10144000644F01003800FFF7F9FE31000500380055
:10145000FFF74CFF0390002D00D1A8E1AB69029388
:101460005D4F31003800FFF7E9FE3100050038001C
:10147000FFF73CFF002D00D19EE1AD692300220063
:101480003C338232643402995D6019606946097B9D
:101490000833507011700232A342F4D1019805F064
:1014A000C9FD009805B0F0BD474F01003800FFF7B7
:1014B000C5FE290006003800FFF718FF0700002EC0
:1014C0002FD03069FFF73EFA2300683320701F7079
:1014D0000023434F290038000093FFF7AFFE290097
:1014E00006003800FFF702FF0700002E1CD030690D
:1014F000FFF708FA2300693360701F70334F29002B
:101500003800FFF79BFE290006003800FFF7EEFECB
:10151000002E00D113E7B369A37023006A3318705B
:1015200010E701235B42D4E701235B420093E5E728
:10153000254F01003800FFF781FE29000600380022
:10154000FFF7D4FE0700002E2DD03069FFF7FAF91F
:1015500023006B33E0701F70214F29003800FFF724
:101560006DFE290006003800FFF7C0FE0700002EC0
:101570001DD03069FFF7C6F923006C3320711F704E
:10158000124F29003800FFF759FE290006003800E5
:10159000FFF7ACFE002E00D1DBE6B36963712300D8
:1015A0006D331870D8E601235B420093D4E7012322
:1015B0005B420093E4E7C046997D0D10B47D0D10A9
:1015C000B77D0D10CB7D0D109D7D0D10B07D0D10E4
:1015D000CF7D0D10697D0D100C7D0D10DD7D0D1082
:1015E000A87D0D107A4F01003800FFF727FE290073
:1015F00006003800FFF77AFE0700002E00D1A1E0B8
:101600003069FFF79FF923006E33A0711F70714F8F
:1016100029003800FFF712FE290006003800FFF706
:1016200065FE0700002E00D190E03069FFF76AF9EF
:1016300023006F33E0711F70674F29003800FFF7F8
:10164000FDFD290006003800FFF750FE002E00D1F6
:1016500080E0B36923722300703318705F4F290054
:101660003800FFF7EBFD290006003800FFF73EFECB
:10167000002E73D0F3685A1E9341637223007133B6
:101680001870574F29003800FFF7D8FD29000600D1
:101690003800FFF72BFE002E64D0F3685A1E9341EA
:1016A000A3722300723318704E4F29003800FFF7E1
:1016B000C5FD290006003800FFF718FE002E55D0A2
:1016C000F3685A1E9341E372230073331870464F38
:1016D00029003800FFF7B2FD290006003800FFF7A7
:1016E00005FE002E46D0F3685A1E93412373230053
:1016F000743318703D4F29003800FFF79FFD290013
:1017000006003800FFF7F2FD002E37D0F3685A1EAE
:1017100093416373230075331870354F29003800E7
:10172000FFF78CFD290006003800FFF7DFFD002ED3
:1017300000D118E6F3685A1E9341A3732300763351
:10174000187013E601235B42009360E701235B42BC
:10175000009371E701235B4200937FE701235B4223
:1017600000938EE701235B4200939DE701235B42D8
:101770000093ACE701235B420093BBE701235B428C
:101780000093CAE701235B4200930BE601235B420F
:1017900000931AE601235B42029600932BE6012395
:1017A0005B42009334E601235B42009341E6012350
:1017B0005B420295009353E601235B4200935DE692
:1017C00001235B42009369E605235B42009368E6D0
:1017D0009D7D0D10A87D0D10B07D0D10BE7D0D10EE
:1017E000C67D0D10E57D0D10A37E0D10AD7E0D1094
:1017F000B47E0D10F0B5050085B000200C0005F09A
:10180000FFFB280005F070FC0190002800D181E169
:101810000100C248FFF7EEF8051E00D13AE1C04FC3
:1018200001003800FFF70AFD290006003800FFF725
:101830005DFD002E00D109E1B36923702300FF3361
:1018400058720023B74F290038000093FFF7F6FCC9
:10185000290006003800FFF749FD002E00D1F8E00E
:10186000F3685A1E934163702300FF339872AE4FA2
:1018700029003800FFF7E2FC290006003800FFF7D6
:1018800035FD002E00D1E8E0F3685A1E9341E37065
:101890002300FF331873A54F29003800FFF7CEFC53
:1018A000290006003800FFF721FD002E00D1D8E006
:1018B000B369A3602300FF3358739D4F290038009C
:1018C000FFF7BCFC290006003800FFF70FFD002ED3
:1018D00000D1CAE02200B369FF32DBB223779074F3
:1018E0006377D074A3771075924F29003800FFF703
:1018F000A5FC290006003800FFF7F8FC002E00D1F7
:10190000B7E02200B369FF32DBB2611CE3775075A8
:10191000CB77A11C9075CB77D075874E290030000E
:10192000FFF78CFC290007003000FFF7DFFC002FD9
:1019300000D1A2E0FB685A1E9341E21CD37723003A
:10194000FF33187601997D48FFF754F80600002F01
:1019500000D19FE023000122794FFF3301009A73E9
:10196000DA731A745A743800FFF768FC3100050006
:101970003800FFF7BBFC0390002D00D181E0AB697C
:101980000293704F31003800FFF758FC310005001A
:101990003800FFF7ABFC002D00D177E0AD692200E5
:1019A00021002300253209315033FF32FF31029EDE
:1019B0005D601E606E46367B0833167050700232D2
:1019C0008B42F4D101996048FFF714F8061E00D14C
:1019D0006DE05E4F01003800FFF730FC310005007C
:1019E0003800FFF783FC0390002D57D0AB690293BA
:1019F000544F31003800FFF721FC3100050038005A
:101A0000FFF774FC002D4ED0AD69220023002100A9
:101A100019322433FF324C31029E5D601E606E46E7
:101A2000367B08335070167002329942F4D1019916
:101A30004748FEF7DFFF051E3DD101235B420093BF
:101A4000019805F0F7FA009805B0F0BD01235B425C
:101A5000F8E601235B42009309E701235B42009310
:101A600019E701235B42009327E701235B420093C0
:101A70003AE701235B4200934FE701235B42009367
:101A800060E701235B42029500937AE701235B4202
:101A9000009384E701235B42009393E701235B42B9
:101AA00002950093A4E701235B420093ADE7012375
:101AB0005B420093BBE7274F01003800FFF7BEFBF6
:101AC000290006003800FFF711FC002E1ED0F36835
:101AD0005A1E934122004C32137091235B00E05454
:101AE0001D4F29003800FFF7A9FB29000600380028
:101AF000FFF7FCFB002EA0D0F3685A1E9341220092
:101B00004D3213702423FF33E05499E701235B42E5
:101B10000093E5E705235B42009394E7F37D0D1006
:101B20005C7D0D103A7E0D10227D0D10187D0D107C
:101B3000407D0D104A7D0D10397D0D10F57C0D1086
:101B4000927E0D100C7D0D105F7D0D10697D0D10C6
:101B50006F7D0D10877D0D107B7D0D107FB5DC2313
:101B60009B0500936C46002302AD01950290154839
:101B70006B60C460144C0668002E07DBA34203D1DF
:101B80000120404204B070BD0133F4E7A342F7D016
:101B90000123836000230669002E03DAA342EFD0FD
:101BA0000133F8E7A342EBD0A02300981B0698422C
:101BB00001D00098E6E7029B002013606B680B6081
:101BC000E0E7C04600002340983A0000F0B5170057
:101BD0008A22434C9200A544079008910EA8002148
:101BE000BFB2099305F08EFD0CAA0BA93800FEF7D1
:101BF000A5FD00260500B0422CD1C02280210B9B00
:101C0000D2051A40C9058A4237D10C9BDC1DE40875
:101C100020000D9405F038FD0925061E1AD001009C
:101C20000DAB22003800FEF799FD051E12D16B4660
:101C3000198C102304930293079B079A3033019366
:101C4000284B40320392009332000D9B0EA8FEF702
:101C500097FD0500300005F021FD002D05D1202263
:101C600009990EA8FEF7ECFC05000EA8FEF7DAFCB9
:101C7000280099239B009D44F0BD1B4A934207D145
:101C80000C9B5C0809230134E4085C433B34BFE748
:101C9000164A934203D10C9BDC082934B8E7144A56
:101CA000934205D103240C9BDB085C435A34AFE715
:101CB000104A934205D103240C9BDB085C434A3451
:101CC000A6E70D4A1B0C1B0493429ED00B4A04004E
:101CD00093429DD10C9BDC1DE4081234640097E70D
:101CE0009CFDFFFF0901202200000170000001603F
:101CF000000002700000026000000370000003603A
:101D00000230800803D001300238FCD1C046C04602
:101D10007047EFF3108072B6704780F310887047F9
:101D2000014B18607047C046E0AD0208044B1B68C9
:101D30001A0008321B68D26F9B181868000E704793
:101D4000E0AD0208054B1B681A0008321B68D26F11
:101D50009B181868000AC0B27047C046E0AD020880
:101D60001D4B98420FD010D840282FD005D80028FE
:101D700030D0102828D019481EE0802828D0802391
:101D80005B009842F7D1144816E0154B984214D0E6
:101D900008D8A0231B0698421CD0124B9842EAD1C7
:101DA000A0200BE0104B98420AD0104B984209D06B
:101DB0000F4B9842DFD10F487047A420C003FBE7C8
:101DC0000D48F9E70D48F7E70D48F5E70D48F3E74B
:101DD0000D48F1E70020EFE706005200FF00520037
:101DE000010000F0090000A0040000F0050000F070
:101DF000030000F0010052000200520003005200F4
:101E000001005000020050000500520070B50A4D5C
:101E100004002B6831331B78834204D8E62107483D
:101E2000490002F087FA2B681A00B0321088444348
:101E3000186A201870BDC046E0AD0208AC800D10D5
:101E400010B50020FFF7E2FF0A4B1C682300B433F3
:101E50001B68C0180368002B0ADB074B1868FFF7E4
:101E60007FFF012263689A609A68002AFCD110BD46
:101E70000248FCE7E0AD020808A802080200500092
:101E80000D4B10B51860002804D0FE235B42038080
:101E900000234380094B1B681A0050321278002A35
:101EA00008D051331B78002B04D0022204490020B3
:101EB00000F086FB10BDC04618A80208E0AD02087D
:101EC000C1A3020870B5C4050500E40D28D102F0D5
:101ED00077FE144B144A1A605D609C60DC60134B03
:101EE0001B6854331978002915D0FFF71FFF040031
:101EF000FFF728FFFA210134013060430C4B0D4CF1
:101F000089004443186805F0F3F90100200005F04A
:101F1000EFF9094BC1188020400005F0F5FD70BDB8
:101F20000648FCE708A802080001001CE0AD020812
:101F300020A1020860F590009808000006005200F9
:101F400070B5C40506000D00E40D2AD1002928D083
:101F500002F036FE144B154A1A605C609E60DD602C
:101F6000134B1B6852331978002915D0FFF7DEFE9A
:101F70000400FFF7E7FEFA210134013060430D4B06
:101F80000D4C89004443186805F0B2F901002000A7
:101F900005F0AEF9094BC1188020400005F0B4FDF2
:101FA00070BD0748FCE7C04608A80208000100050C
:101FB000E0AD020820A10208C0EA21014826000085
:101FC0000600520070B506000C001500072903D961
:101FD0001449154802F0AEF91F232A009A4303D092
:101FE0001249114802F0A6F9114B1B689A695B6906
:101FF000B01AC0090001C0181F231D40032C07D8C8
:10200000E400A340A54002689A431543056070BDF3
:10201000043CE400A340A54042689A431543456050
:10202000F5E7C046910200005E810D1092020000AB
:10203000E0AD0208F0B585B000900D001400002856
:1020400000D138E1002A00D135E1072903D94E211A
:102050009A4802F06FF92368012B03D94F21974862
:1020600002F068F90F2362689A4303D05021934825
:1020700002F060F91F22237A934303D051218F4845
:1020800002F058F9E368032B03D952218B4802F080
:1020900051F92369012B03D95321884802F04AF9E9
:1020A0006369012B03D95421844802F043F9A369E1
:1020B000012B03D95521814802F03CF9E369032B38
:1020C00003D956217D4802F035F9236A012B03D943
:1020D00057217A4802F02EF9636A012B03D958215F
:1020E000764802F027F9A36A012B03D959217348D6
:1020F00002F020F9E36A032B03D95A216F4802F05A
:1021000019F9236B072B03D95B216C4802F012F9F4
:102110002668072D04D9CC216948890002F00AF904
:102120000122AA400192012E07D96649644802F0B3
:1021300001F9009B019A9A6004E0002EF9D1009BFE
:10214000019A5A606668072D03D95F495C4802F01E
:10215000F1F80F2332009A4303D05C49584802F04B
:10216000E9F80F215A4FAB0002933B6808007D331A
:102170001A78009B0E40D2181368A9009C46AB0049
:10218000984063468E4083431E431660227A29009E
:102190000098FFF717FFE668082D03D94D49484816
:1021A00002F0C8F8032E03D94B49454802F0C2F8A3
:1021B000032108006B0003933B686F00B8400E409A
:1021C000BE407C331A78009B9A18136883431E43E1
:1021D00016602669082D03D94049394802F0AAF84B
:1021E000012E03D93E49364802F0A4F8019A009B1B
:1021F000D74301221640AE409B693B401E43009BE3
:102200009E616669072D03D936492D4802F092F880
:10221000012E03D934492A4802F08CF801202C4BB6
:1022200006401968AE400B0084467E331B78009A46
:10223000D3181A68174037431F600B0062467F337C
:102240001878009B6E001818A36910361340AB4035
:10225000E56902321540B540B2402B43019D076845
:102260002A4397433B4303600220042580310A78C8
:10227000009B9A18636A11685B000340A06A8000A3
:10228000284003436046256A284018250343E06A36
:10229000C00028400343206BFF244001204003433B
:1022A000FE20029D80000540AB400020A1430B436F
:1022B000136005B0F0BD0D48FBE7C04607810D1067
:1022C0005E810D1031030000CD030000CE0300003D
:1022D000E0AD0208F1060000F20600007206000000
:1022E000730600000C0400000D04000001005A00F9
:1022F0000B4B70B51B680500B4331B680C00C3188A
:102300001B68002B09DA0B0C03D00649064802F0C3
:1023100011F80020A4B26C6070BD0448FCE7C04610
:10232000E0AD0208DE020000AC800D1001008A0062
:10233000036870B505000C00002B0BDAC2600B0CB3
:1023400004D0B1210448890001F0F4FF0020A4B2B8
:10235000AC6070BD0148FCE7AC800D1001008A0044
:1023600070B505000C1E03D1A221084801F0E2FF60
:10237000074B1B68B4331B68EB181B68002B03DA90
:102380000020EB68236070BD0248FCE7B6810D10A9
:10239000E0AD020801008A00024B1A68002A00D151
:1023A000186070471CA80208F0B5314D1F002B685B
:1023B00085B0040002910392002B03D1BE212D4869
:1023C00001F0B8FF2C23FF225C432B683D001C1951
:1023D0003B0A3F0CA760284F134063603B681540E1
:1023E000256031331B789D4204D3E6212348490000
:1023F00001F0A0FF3B681A00B032128855431A6AF8
:102400003233AD1825611B7865689D4204D3F421F1
:102410001A48490001F08EFF3B681E6A2B0080338A
:102420005B01F3186361A36801931B0C09D0134F80
:102430001349380001F07EFF82213800890001F045
:1024400079FF019B6D011B041A0C13430D4A75198A
:10245000AD182B60039BE361029B23620023A36101
:102460000A9B002B01D01B88A38105B0F0BDC0469C
:102470001CA8020810820D10E0AD0208AC800D10FF
:102480000702000008100000F0B5040085B0002825
:1024900003D15B21214801F04DFF6368032B03D971
:1024A0005D211E4801F046FFE36A002B03D1612144
:1024B0001A4801F03FFF236B002B03D1622117481C
:1024C00001F038FFA36802AD2B80154B22681B6812
:1024D000E16ADB8EE0689B18AB706368A26A0393C5
:1024E00000952369266A676AFFF75EFF00213B00BB
:1024F0000A0000913000FFF757FF216B280001F020
:10250000A1FE0022AB5E002B06DB1F2213401E3A09
:102510009A401300034A136005B0F0BD10820D10FD
:10252000E0AD020800E100E0F7B504000F00151E61
:10253000019304D183211D48490001F0FBFE1C4E8C
:102540003368002B04D108211848FF3101F0F2FE56
:102550002C235C4332685F4314192669D719002E77
:1025600020D0BB69002B1FD13368002B1CDA01225D
:102570006368140011009C407B6899402B68090433
:102580009BB20B432B60019BF5607B62BA61230C0D
:1025900004D0B1210748890001F0CCFE0020A4B28C
:1025A000B460FEBD0448FCE70448FAE710820D1051
:1025B0001CA80208AC800D1004028A0007028A00E1
:1025C000F8B5114F04003B680E001500002B04D134
:1025D00068210E48FF3101F0ADFE2C2060433C68BD
:1025E0002418236A002B04D16C210848FF3101F024
:1025F000A1FEE369AB4204D90020236AAD00EE508E
:10260000F8BD0348FCE7C0461CA8020810820D1064
:102610000A028A00002373B504000193984204D192
:10262000ED212C48490001F085FE2369002B04D1DF
:10263000DC212848FF3101F07DFE6369002B04D1C5
:10264000EE212448490001F075FE236A002B04D1D5
:10265000DE212048FF3101F06DFE6269D5682B0C48
:1026600022D01B04136013681B4B20691B68B43312
:102670001B68C3181B68002B16DA01A9FFF770FE50
:102680000026B0420CD10198E26903681E0CDBB24F
:102690009A4205D9226A9B009B58002B00D098478C
:1026A00031002069FFF724FEADB2002D09D0636927
:1026B0001D6000251B68636AAB4205D098476562C0
:1026C000A56163691B6873BDA36A002BF8D09847A6
:1026D000F6E7C04610820D10E0AD020870B5084C58
:1026E00005002368002B04D1DD210648490001F0D4
:1026F00021FE2C20454320684019FFF78BFF70BD59
:102700001CA8020810820D1070B50A4D04002B6839
:1027100031331B78834204D8E6210748490001F091
:1027200009FE2B681A00B03210884443186A20183A
:1027300070BDC046E0AD0208AC800D10F8B5174B77
:102740000D001B6831331B78834225D9002923D023
:102750001F240B681C401FD1FFF7D6FF07002B6812
:102760000F4EDA0821003060686804F0CBFF2100CA
:102770003800FFF7BDFD21002A003068FFF7D8FDC3
:10278000041E07D101003068FFF7B2FD03002000EE
:10279000002B00D00348F8BD0348FCE7E0AD020879
:1027A00020A8020801018A0003018A00F7B5184F2A
:1027B00004003B680191DE683368834226D9002516
:1027C000A94202D1FFF7A5FA050038680368002B7B
:1027D0001ADA1F2201232240934064097268A40080
:1027E0001419226813420DD09A432260002400215C
:1027F000FFF77EFD019B002B02D12800FFF78DFA29
:102800002000FEBD034CF2E7034CF3E7034CF7E76F
:1028100020A80208020188000301880004018A0040
:102820000A4B1B68DB681A6882420DD959681F235E
:10283000420918401E3B8340920050581840431EE6
:102840009841034BC01870470248FCE720A80208D3
:102850000001880004018A0070B5154E0400336839
:102860000D009B6CC340DB0703D4A721114801F086
:1028700061FD0F2D03D9A8210E4801F05BFDF02268
:102880002B041203290013400F2211400B4331681F
:10289000A402096964188021C9016350605810407E
:1028A000401B431E9841044B4042184070BDC04637
:1028B000E0AD02086B820D100300C20070B5094D37
:1028C00004002B689B6CC340DB0703D4C721064878
:1028D00001F030FD2B6810341B69A402E0580F236F
:1028E000184070BDE0AD02086B820D1070B5040099
:1028F0000D00002804D17A212448FF3101F01AFD8F
:102900006B89DB0B04D0BD212048490001F012FD8A
:102910000222AB799343012B04D07C211B48FF3169
:1029200001F008FD0222EB799343012B04D0BE2174
:102930001648490001F0FEFC6A897F231100994383
:1029400022D10721AB7952020B4013436A7A31310D
:1029500092071343EA79D2000A4013430122297AED
:102960004A40920113431A0009490A409A420BD186
:102970006262606A0840801A43425841054B4042F7
:102980001840054BC01870BD0448FCE76B820D1061
:10299000DBFEFFE0FDFF3DFF0300C2000100C200BF
:1029A00070B504000D00002804D1C2212E48FF316B
:1029B00001F0C0FC6B89DB0B04D0E1212A484900FF
:1029C00001F0B8FCAB79072B04D9C4212648FF31AC
:1029D00001F0B0FCEB79072B04D9E2212248490031
:1029E00001F0A8FC2B79073B182B04D9C6211E48FF
:1029F000FF3101F09FFC6B897F22190091430A1E71
:102A00002ED12968FF3291430A006979A8790A43D7
:102A100007215B02084018436B7A31319B0718434A
:102A2000EB79DB000B4018430123297A4B40F82156
:102A30009B0118432B7949051B060B400343636038
:102A40002260216891420DD16068084A1040C01A86
:102A500043425841064B40421840064BC01870BDD7
:102A60000548FCE70348FAE76B820D10FFFEFFFF05
:102A7000FDFF3DFF0300C2000100C20010B5041EAF
:102A800004D1FF210748490001F054FC8023626A09
:102A90001B0613436362606A034BC00F0138184082
:102AA00010BDC0466B820D100300C20010B5041E9D
:102AB00003D10749074801F03DFC802362681B06EB
:102AC000134363606068044BC00F0138184010BDA9
:102AD0004E0200006B820D100300C20070B50400AE
:102AE0000D00002803D12449244801F023FC0222D0
:102AF000AB799343012B04D0A5212048C90001F0F4
:102B000019FC0222EB799343012B03D01C491B488B
:102B100001F010FC1B4B1B682F331A78012A26D1B9
:102B200069897F230800984323D10720AB794902A4
:102B300003400B43697A313089070B43E979C900B7
:102B400001400B43297A4A40920113431A000E496F
:102B50000A409A420DD16262606A0840801A43427C
:102B600058410A4B40421840094BC01870BD0948F3
:102B7000FCE70948FAE7C046270500006B820D1004
:102B800029050000E0AD0208DBFEFFE0FDFF3DFF90
:102B90000300C2000200C2000100C20070B50500BF
:102BA0000C00002803D12F492F4801F0C3FBA37963
:102BB000032B03D92D492C4801F0BCFBE379032BEF
:102BC00003D92B49284801F0B5FB2379073B182B83
:102BD00004D9AF212448C90001F0ACFB254B1B6888
:102BE0002F331A78012A36D161897F230800984350
:102BF00033D10720A379490203400B43617A313076
:102C000089070B43E179C90001400B43217A4A400F
:102C1000F821920113432279490512060A40134311
:102C20001A0015490A409A4217D1FF232068984399
:102C3000030060796A6003432B60286898420ED1D4
:102C400068680840801A434258410C4B4042184083
:102C50000B4BC01870BD0B48FCE70B48FAE708485F
:102C6000F8E7C046750500006B820D107605000080
:102C700077050000E0AD0208DBFEFFFFFDFF3DFF32
:102C80000300C2000200C2000100C20010B5041E11
:102C900003D10B490B4801F04DFB0B4B1B682F3345
:102CA0001B78012B0AD18023626A1B0613436362DF
:102CB000606A064BC00F0138184010BD0448FCE79D
:102CC000BD0500006B820D10E0AD02080300C200DC
:102CD0000200C20010B5041E03D10B490B4801F0DD
:102CE00029FB0B4B1B682F331B78012B0AD1802348
:102CF00062681B06134363606068064BC00F0138AF
:102D0000184010BD0448FCE7160600006B820D1049
:102D1000E0AD02080300C2000200C20070B504006A
:102D20000D00002803D12149214801F003FB2B7835
:102D3000032B03D91F491E4801F0FCFA6B78032BC3
:102D400003D91D491A4801F0F5FA1C4B1B682F33B3
:102D50001A78012A26D1A9887F230800984323D115
:102D600007202B78490203400B43E978313089076B
:102D70000B436978C90001400B43A9784A4092018E
:102D800013431A000E490A409A420DD16262606AEA
:102D90000840801A434258410A4B404218400A4BAF
:102DA000C01870BD0948FCE70948FAE7560800005A
:102DB0006B820D105708000058080000E0AD0208B3
:102DC000DBFEFFE0FDFF3DFF0300C2000200C2008A
:102DD0000100C20070B504000D00002803D1214994
:102DE000214801F0A7FA2B78032B03D91F491E486D
:102DF00001F0A0FA6B78032B03D91D491A4801F0A2
:102E000099FA1C4B1B682F331A78012A26D1A988FE
:102E10007F230800984323D107202B7849020340E1
:102E20000B43E978313089070B436978C9000140C9
:102E30000B43A9784A40920113431A000E490A40F5
:102E40009A420DD1626060680840801A434258413E
:102E50000A4B404218400A4BC01870BD0948FCE7B5
:102E60000948FAE7A70800006B820D10A8080000C7
:102E7000A9080000E0AD0208DBFEFFE0FDFF3DFF1A
:102E80000300C2000200C2000100C20010B5041E0F
:102E900003D10B490B4801F04DFA0B4B1B682F3344
:102EA0001B78012B0AD18023626A1B0613436362DD
:102EB000606A064BC00F0138184010BD0448FCE79B
:102EC000EB0800006B820D10E0AD02080300C200A9
:102ED0000200C20010B5041E03D10B490B4801F0DB
:102EE00029FA0B4B1B682F331B78012B0AD1802347
:102EF00062681B06134363606068064BC00F0138AD
:102F0000184010BD0448FCE7440900006B820D1016
:102F1000E0AD02080300C2000200C20070B5040068
:102F20000D00002803D12149214801F003FA2B7834
:102F3000032B03D91F491E4801F0FCF96B78032BC2
:102F400003D91D491A4801F0F5F91C4B1B682F33B2
:102F50001A78012A26D1A9887F230800984323D113
:102F600007202B78490203400B43E9783130890769
:102F70000B436978C90001400B43A9784A4092018C
:102F800013431A000E490A409A420DD16262606AE8
:102F90000840801A434258410A4B404218400A4BAD
:102FA000C01870BD0948FCE70948FAE7A809000005
:102FB0006B820D10A9090000AA090000E0AD02080B
:102FC000DBFEFFE0FDFF3DFF0300C2000200C20088
:102FD0000100C20070B504000D00002803D1214992
:102FE000214801F0A7F92B78032B03D91F491E486C
:102FF00001F0A0F96B78032B03D91D491A4801F0A1
:1030000099F91C4B1B682F331A78012A26D1A988FD
:103010007F230800984323D107202B7849020340DF
:103020000B43E978313089070B436978C9000140C7
:103030000B43A9784A40920113431A000E490A40F3
:103040009A420DD1626060680840801A434258413C
:103050000A4B404218400A4BC01870BD0948FCE7B3
:103060000948FAE7F90900006B820D10FA0900001F
:10307000FB090000E0AD0208DBFEFFE0FDFF3DFFC5
:103080000300C2000200C2000100C200094B1B681D
:103090002F331B78012B0AD18023426A1B0613436E
:1030A0004362406A044BC00F013818407047034820
:1030B000FCE7C046E0AD02080300C2000200C20007
:1030C000094B1B682F331B78012B0AD180234268E0
:1030D0001B06134343604068044BC00F013818407F
:1030E00070470348FCE7C046E0AD02080300C20099
:1030F0000200C200036810B50400002B07D00120B5
:1031000001F00EF92368013B2360002B01D0002061
:1031100010BD0148FCE7C0460200B200030A087077
:103120004B70030C000E8B70C870704770B50400B4
:103130000D00002841D000293FD0002B3DD05A621D
:10314000F9220321D20083588B4383502B68DBB2D2
:10315000012B03D957311A4801F0ECF8AB68DBB208
:10316000032B03D95B21164801F0E4F86B68072BA9
:1031700003D95C21124801F0DDF8EB68DBB2012BCA
:1031800003D95D210E4801F0D5F8C022E021AB68DB
:1031900092011B0313406A68C90212040A401343D8
:1031A0000122296800200A4080211343EA6849046B
:1031B00012060A401343236070BD0248FCE7C04674
:1031C000C2820D100400B20010B50400012907D915
:1031D000A021074801F0AEF801232268134304E060
:1031E0000029F9D1012203689343236010BDC04632
:1031F000C2820D1070B54E1EF3B204001500012BF3
:1032000007D9042925D0082927D0E521154801F040
:1032100091F8032D03D9E621124801F08BF8072E0F
:1032200014D8300004F05AF8041312171212121BAB
:1032300080231B01E418002C08D0C0222D04920228
:1032400023681540084A13401D43256070BD88233C
:10325000EFE7032ADFD89023EBE7032ADBD8982394
:10326000E7E7C046C2820D10FFFFFCFFF0B5160075
:1032700089B005930EAB04CB01901B7802910493A7
:1032800010AB1D78331FDBB20392129CFA2B04D8CB
:103290003E213B48FF3101F04DF8049B043BDBB27B
:1032A000FA2B04D89F213648490001F043F86B1EE1
:1032B000012B08D9FB222B1F134204D04021304898
:1032C000FF3101F037F8119B2D02DF07039B360415
:1032D000002B46D0059B002B04D1A0212848490093
:1032E00001F028F8049BFF2B04D142212448FF3130
:1032F00001F020F8F0231B011D40636A0793C023EF
:103300009B021E40029B2B4333433E0C00270024AC
:10331000C0221F43019B20001F650727049B9202C8
:103320001B0413401D43039B9C4202D2154B984241
:1033300001D109B0F0BD019B5B6C3B40032B0CD865
:10334000059B03991B5D01342B4332008C4200D254
:1033500000221343019AE4B2136507A8FFF7CAFEDF
:10336000E1E7F0231B011D40636A3F0C0793C02374
:103370009B021E40029B2B4333433E00C7E7C046DF
:10338000C2820D100200B200F7B50193043BDBB21C
:1033900005000F001600099CFA2B04D8D521164809
:1033A000490000F0C7FF002E21D007226B6C1340AC
:1033B000032B1ED88023C021721EDB0292B21A4357
:1033C000019B89021B040B4013432B65381E0DD053
:1033D000089B2760F922A660E36102230020A36115
:1033E000D200A958013B0B436660AB50FEBD0348B9
:1033F000FCE70348FAE7C046C2820D100400B200A1
:103400000100B200F7B50193043BDBB205000F00E9
:103410001600099CFA2B04D89C211648890000F05C
:1034200089FF002E22D007226B6C1340032B1FD87C
:103430008023C021721E92031B03920B1A43019B2F
:1034400089021B040B4013432B65381E0DD0089BCB
:10345000E760F9226661236204230020A361D200A1
:10346000A958023B0B432661AB50FEBD0248FCE766
:103470000248FAE7C2820D100400B2000100B20057
:10348000F0B51F00043BDBB28FB006000D00140046
:10349000FA2B03D85B495C4800F04CFF002C00D1AC
:1034A000ABE00722736C1340032B00D9A7E0631E27
:1034B0009B039A0B80231B031343C0223F049202F9
:1034C00017401F433765281E0ED0149B00205B6AEF
:1034D00007950393042309940C900A930A9B042BE9
:1034E00002D14A4B984201D10FB0F0BD099B079C15
:1034F00000933300C43301931D680F231D40009BCC
:103500009D4200D91D00002D17D1009B07940993FF
:10351000002B0CD1F92202210320D200B3588B4397
:10352000B3500A900C9B002B01D00C9B9847009B3A
:1035300003A80993FFF7DEFDD0E7082D0AD1370075
:10354000D83738682100FFF7E9FD3868211DFFF7FB
:10355000E5FD05E0012D09D13300D0331B68237050
:10356000009B64195B1B0093019BC5E7022D06D1EC
:103570003300D4331B6823701B0A6370F0E7032DFC
:103580000AD13300D4331B6823701B0A63703300E5
:10359000D0331B68A370E3E73700D83738682100C1
:1035A000042DD4D0052D06D1FFF7B8FD3300D0335C
:1035B0001B682371D4E7062D08D1FFF7AFFD330058
:1035C000D4331B6823711B0A6371C9E7072D0CD123
:1035D000FFF7A4FD3300D4331B6823711B0A63710A
:1035E0003300D0331B68A371BAE7FFF797FD386843
:1035F000211DFFF793FD0825B2E7054874E705484C
:1036000072E7C046CD020000C2820D100200B20077
:103610000400B2000100B20000290CD00722436C64
:103620001340032B09D8C023013989B21B03194366
:103630000165002070470248FCE70248FAE7C046EF
:103640000400B2000100B20000230B604B608B60ED
:103650000B61CB604B618B61802302681B061343B7
:103660000360704730B58B6987B0DB680C001500CC
:10367000002B0FD019681A79012303932378C9B25C
:103680000293FF230193002304950093FFF7EEFDBF
:1036900007B030BD0048FBE78000B20070B51600EF
:1036A00000220400080086B00A9D039204951900C8
:1036B000037800920293FF23200001931300FFF789
:1036C000D5FD002806D1030000950122310020001D
:1036D000FFF7D6FE06B070BD30B50F24012385B0CC
:1036E0008D696C442370AB6A002B0BD01B68009271
:1036F000DBB22200FFF7D2FF002803D12378AA6BA8
:10370000134023702078431E9841C0B205B030BDED
:10371000F0B587B017000C9A05000C001E00FFF7EB
:10372000A1FF002812D1A3690122DB6B022B00D07C
:103730001300039222780C990292002204910093C4
:1037400001923B0031002800FFF790FD07B0F0BD6B
:103750000023F0B58F6989B00D00F96A07AC060047
:103760000292238099425FD03A6B9A425CD0BB6A46
:10377000002B59D01B68096812680593029BC9B2D7
:1037800003910492009322000B002900FFF786FFAB
:1037900000282FD16B46FF6B1B7C0493402F1ED05B
:1037A000802F29D0022F41D16B46029A1B7D290020
:1037B000009230002200FFF771FF00281AD10D227D
:1037C000029B04A900935218039B29003000FFF7C5
:1037D00065FF00280ED163781F43677002E02378ED
:1037E0001F4327702200029B0093049B2900300096
:1037F000FFF78EFF09B0F0BD0D22029B04A90093D4
:103800005218039B29003000FFF748FF0028F1D130
:10381000802362785B4213430D226370029B04A9EC
:1038200000935218049BE1E70148E3E70148E1E710
:103830008000B2000300B200F0B51F008B6989B0B0
:103840001C6A0500002C47D0002A47D0586A0E9EFB
:10385000B04243D34869C6B24869002800D10E7807
:1038600021682079C9B2079110990296049100212C
:103870000391617901911B6807990093130002007D
:103880002800FFF7F3FC002824D1A1684B1C12D1BB
:103890002169002904D02800FFF7BEFE002819D1B5
:1038A000109A237D01920F9A3900009228000E9AF7
:1038B000FFF76AFD0EE0109B227B0493FF23039029
:1038C000019300900300C9B202962800FFF7CEFCD6
:1038D0000028DDD009B0F0BD0148FBE70148F9E759
:1038E0008000B2000400B200F0B5CDB006000C1E9E
:1038F0000692089303D1C449C44800F01BFD00237D
:103900000BAF656B3B80BB70089A06993000FFF7E0
:1039100071FC002D03D1BE4A10004DB0F0BD2B68E4
:103920002A79D9B2529B3000049300230393069B5B
:1039300002936B790193032300933B00FFF796FCFE
:10394000021EE9D129693000FFF766FE021EE3D1AD
:1039500052992B7D0CAD01910090FF32290030006F
:10396000FFF750FD021ED7D1529B5E6AA94B5299B8
:103970008869032812D09A42CED0002E0CD00120A4
:10398000013E00F0CDFC3200531E9A41A24B524240
:103990001A40A04BD218E9E73200E8E7002ABBD171
:1039A0002B78532BB7D16B78462BB4D1AB78442B03
:1039B000B1D1EB78502BAED12B79052BABD96B79EC
:1039C000012BA8D1297BA3686D18AD7806956D08E9
:1039D0000540012D00D8B1E0022D00D1ADE00F254A
:1039E0001F278E080936B6004CA880190138FF3809
:1039F0000068BC46054001356D00079505093D404E
:103A0000079F01356F4309970327400A3840834DCC
:103A10004000405B099D45430DA8256485596646D5
:103A2000280E3040079E013070436E0F37407C4EA9
:103A30007F00BE5B40277043606460462E0A0640EC
:103A400010382840AD0400D4383F01304000013622
:103A500046437E430CA8A6640E1D87197D78079007
:103A60002802FD782D0605430798865D3543BE780C
:103A70003604354364D40135ED080798656047186E
:103A80003D0028352E78012528003609B0403E7FBC
:103A90006062B5400698A5610CAD800655D502263A
:103AA0000898B043012850D0082084467F7A8C447F
:103AB0001F60002760461F71079F5E713F5C7F0992
:103AC0005BD1033E9E6060461F262D5C35401D6124
:103AD00002251D750623E56804262B6000232B7143
:103AE000256907982E602B71E5695C362E602B7175
:103AF0004118487F6569022728602B716B71012589
:103B0000266A01206D42337137607371B56033618D
:103B100033750526A063A06A3A310660266B0371EF
:103B2000337108784006400F052800D9F4E6E16AB1
:103B300003F0D4FB65787E847878042020604EE71B
:103B40008026033D3606354397E70698400618D58C
:103B500002260898B043012813D00A2084466E1824
:103B6000F67A8C441E60002660461E715E712F5CE2
:103B70007F09B74201D1013EA4E7FF271E739F6072
:103B8000A1E710270698074017D06E18F67B012092
:103B90001E600F00002658711E710E37EE5D76090B
:103BA00007D1013E9E60ED5D1F2635401D61012558
:103BB0008FE7FF2618739E60F5E7012606983040D0
:103BC00014D00C2084468C4460466E18767B1F719E
:103BD0001E605F712E5C760904D1013E9E606046D6
:103BE0002D5CE1E7FF261F739E60F8E703251D604B
:103BF000043D187158719D60186118756AE7E56396
:103C000035600D6088E6C046F90300002A830D1078
:103C10000500B2000200B200FEFF4DFF1A830D1036
:103C200022830D100123E763336034330B6073E6A6
:103C30004023E3633F3B33600433F7E78023E363D0
:103C4000423B33600133F1E7F0B589B0029007924F
:103C5000002800D11EE1002900D11BE14B6805932B
:103C6000002B00D116E1002A00D113E10B68069366
:103C7000002B00D10EE10023C02603930493B6026B
:103C8000039B059A9B00D458002C4DD023785A1ED4
:103C9000012A09D90422043B9343DBB2002B03D051
:103CA0006E217D4800F046FB237A032B03D96F2158
:103CB000794800F03FFBA369002B03D170217648BF
:103CC00000F038FBA3691B68013B032B03D971216A
:103CD000714800F02FFB2278501E072800D9D7E04A
:103CE00003F0FCFA0432D635D6D6D6388021029BB2
:103CF00009015D18237A2968684F1804304039405B
:103D00000143042029606168014226D00799029886
:103D10000091A169FFF7E8FD00281ED00823039A4F
:103D20009340049A1A430492039B01330393039A2A
:103D3000069B9342A4D10020049B002B02D0B2200A
:103D40000004184309B0F0BD029B8821D0E7029B14
:103D50009021CDE7029B9821CAE763689B07E3D5D2
:103D60002169E06803F04AFB002903D08C214A480E
:103D700000F0E0FA23694A4A934202D95A1E1342DC
:103D800003D08D21444800F0D5FAFF218C466746C8
:103D9000E168A069B9438268036AA9602169494260
:103DA000B943E96001680320013901406069471E99
:103DB000B841000201432962002A2DD01068002179
:103DC000471C08D067460740802011790006090487
:103DD00031400743394329645179906809043140DF
:103DE00069640021471C07D08027117BC0B20904F9
:103DF0003F063140384301430020A96411698142E4
:103E000005D01F3001390140802000060843E864D6
:103E1000127D120432402A65002B2CD01968002232
:103E2000481C07D080201A79C9B21204000632401B
:103E300001430A432A665A799968120432406A6635
:103E40000022481C07D080201A7BC9B21204000649
:103E5000324001430A430021AA661A698A4205D00A
:103E60001F31013A0A40802109061143E9661B7D92
:103E70001B0433402B6702216268FF31114080220E
:103E8000237A12061B0433400A4313432B604BE78B
:103E9000044851E7034855E72A830D10FFFFFCFF54
:103EA000FFFF00000400B200104B1B683C331B787E
:103EB000834219D9042910D94B1EFF3B132B13D869
:103EC0001F2319400A4B8000C018C02304229B0006
:103ED000C1504033C250002070470723D0301940F2
:103EE000034B8000C150F6E70248F5E7E0AD020859
:103EF0000000264001004A0010B50F4B04001B686B
:103F00003C331B78834204D8A3210C48490000F0BD
:103F100011FA0B4BA400E418D0239B00E0580723B0
:103F20001840042807D1C0239B00E0581F230340FA
:103F300080204000184310BDE0AD020889830D10B9
:103F400000002640F7B5041E03D14649464800F05C
:103F5000F1F9B023454DDB00EB58002B00DA7FE090
:103F6000434B22689A4203D942493F4800F0E2F9A4
:103F7000E2792368511E8A419B0312069B0B13436F
:103F8000B022D200AB50A3883B4FBB4204D994214E
:103F90003548890000F0CEF92389384EB34203D961
:103FA0003749314800F0C6F92389A28835491B04F6
:103FB000D204D20C0B401343334AAB50A37A019185
:103FC0000F2B04D996212848890000F0B3F9E37A31
:103FD0000F2B03D92D49244800F0ACF9A389BB422B
:103FE00003D92B49204800F0A5F9FF22E37A29499B
:103FF0001B011340A28912020A400F211343A27A27
:104000000A40C0211343A27B890512070A401343CB
:10401000B122D200AB50A379042B03D91E49124818
:1040200000F088F9238AB34204D999210E48890007
:1040300000F080F9E020A379184AC0001B02A958BB
:104040000340174801400B43AB50238A01981B04DF
:10405000A95803401348014000200B43AB50FEBD5C
:104060001148FCE73F02000089830D100000264044
:10407000FFFF030049020000FF1F0000FF010000D6
:10408000510200000000FF018405000059020000F9
:104090005A02000000FF1F00630200008C050000B0
:1040A000FFF8FFFFFFFF00FE03004A00F7B5802284
:1040B000B22607000500324B324C1206E158F600DA
:1040C0000A43E25000930422A359134201D1002D68
:1040D00035D1B1208023C00022582B499B050A40CE
:1040E000134323500191002F01D0002D06D0B022A0
:1040F0008023D200A1581B060B43A3500126B223F4
:10410000DB00E358334224D1002D1DD1002F24D0F1
:10411000B121C9006258019B1C481A4080239B05AD
:104120001343B0226350D200A3585B005B08A35036
:10413000009B009AE3585B005B08A350FEBD012082
:1041400000F0EEF8013DBEE7300000F0E9F8013D77
:10415000D5E7002F01D0002DDAD0B122C0230020F6
:10416000D200A1589B050B43A3508742E6D0681E9E
:1041700085416842064D054B2840C018DEE7C04621
:104180008C05000000002640FFFFFFCF02004A0020
:10419000FEFFB5FF70B51A4E050033680C001A001B
:1041A00028321278012A15D182080721100088438D
:1041B0000FD103202840C00084401B6892002033A8
:1041C0009B182200FF24844019684A4014404C4048
:1041D0001C6070BD5B8FDBB28B4203D17F2109482D
:1041E00000F0A8F807208022054080203368920163
:1041F0001B680006A4180543A400E550E9E7C04683
:10420000E0AD0208E2830D100A4B70B59B680A4EC0
:1042100010300D008400B34209D1002904D1A0213F
:104220000648490000F086F83059355170BD044BFE
:104230001859FBE700ED00E000A00208E2830D1032
:1042400000000D10F8B506000D00002841D04368AD
:10425000032B03D93B21204800F06CF80023F05ECB
:10426000002828DBB178FFF795FF0024FF22032701
:1042700094460023F05E716883B21F40FF006646DB
:10428000BA4089013140D243B940002815DB134EB2
:1042900083089B009B19C026B6009F593A401143E2
:1042A00099510F4B9A680F4B9A4202D12900FFF7A0
:1042B000ABFF2000F8BD0C4CD8E70F263340083B7D
:1042C000074E9B089B009B19DE6932401143D96160
:1042D000E7E7054CEDE7C046E2830D1000E100E0A2
:1042E00000ED00E000A002080100560070B5802536
:1042F00004002D02AC4205D8064B18686043FDF758
:10430000FFFC70BD044B1868FDF7FAFC034BE41882
:10431000F0E7C04630A1020828A102080080FFFF94
:1043200010B5034B1B785843FDF7EAFC10BDC0469F
:1043300034A1020870B50D00044C010018222000C1
:1043400003F0D3FAA56101BEFEE7C046B0A702089C
:104350008022054B12069A64986C044BC043C01728
:104360001840034BC018704700002740FDFFB9FFFD
:10437000030046008022054B120198585B68DBB2AF
:10438000002B02D08023DB02184370470000264038
:10439000FEE7000002680A4B10B5DA6142681A6253
:1043A00082685A62C2689A620269DA6242691A6372
:1043B00082695A63C2699A63FFF7EAFF10BDC0467B
:1043C000B0A70208F0B51922002800D14B322A4BC1
:1043D0008A4292411B6852421C00A83424881D68FE
:1043E000671903253E68AE4316433E601E68A41954
:1043F0002768224E374027601C00AA3424881E6894
:10440000A7193E68AE4332433A601A681B4EA218A1
:1044100014682640166000280ED00020102904D908
:10442000213088428041404201300F225B68196888
:10443000914308431860F0BD1A00553212788A4241
:10444000F3D21A005632127801208A42EDD21A00B5
:104450005732127800188A42E7D21A00583212787E
:1044600028008A42E1D21A005932107888428041ED
:1044700040420430D9E7C046E0AD0208FFFCFFFF30
:10448000B0235B055A782120002A01D05878C0B2A9
:104490007047B0235B059A89002A02D0988980B2C0
:1044A000704780204000FBE770B5FFF7F2FF8023E4
:1044B000184A5B00984215D111680F240B000222A4
:1044C000983318680B6818180368A34313430360F4
:1044D00008009C300B6801685B181968A1430A4307
:1044E0001A6070BD1268B0201100C02598311468A0
:1044F0000968094B4005C35861180C68AD002B438F
:1045000023430B6011009C3113680A689B18034A0F
:104510008258E5E7E0AD02084818000044180000A2
:1045200070B5FFF7B6FF8023184A5B00984215D19B
:1045300011680F240B000322983318680B681818B1
:104540000368A3431343036008009C300B680168B1
:104550005B181968A1430A431A6070BD1268B02441
:104560001100C120C0269831156809686405400112
:10457000235869180D68B60033432B430B601100B4
:104580009C3113680A689B182258E5E7E0AD0208E1
:1045900010B5FFF77EFF8023114A5B0098420DD1D2
:1045A000136810491A00983212681B689B181A6821
:1045B0001140C022D2010A431A6010BDB021126816
:1045C000094B4905CB581100C02098310968126881
:1045D00080005218116803430B431360EDE7C04697
:1045E000E0AD0208FF8FFFFF1818000070B5FFF75D
:1045F00050FF8023144A5B0098420DD11368134981
:104600001A00983212681B689B181A6811408022A1
:10461000D2010A431A6070BD1268B0241100C0268E
:10462000983115680A4809686405235869180D68A7
:10463000B60033432B430B6011009C3113680A68AA
:104640009B182258E6E7C046E0AD0208FF8FFFFF47
:104650004C18000010B50020FEF730F90400FFF7F9
:104660000FFF01221300222801D863426341134047
:10467000180010BD10B5074C236831331B78002B90
:1046800004D1E62104484900FFF754FE2368186A64
:1046900010BDC046E0AD0208AC800D1030B504007E
:1046A00085B00D00042803D927492848FFF742FEAA
:1046B0006B1E012B07D9FB222B1F134203D0244969
:1046C0002248FFF737FE234BA400E458042D01D005
:1046D000012D1AD100200FE0A3682B420BD1E36813
:1046E00029001A685B6802920193039302A8236869
:1046F0009847194B1C606469002C04D0174B9842F2
:10470000EAD1012DE8D105B030BD022D06D1124B02
:104710001B68181EF7D01C6903E01C006369002B9E
:10472000FBD10020002CEED0A3682B4209D1E36816
:1047300029001A685B6802920193039302A8236818
:1047400098472469EEE7C046E50900003B840D1058
:10475000E609000048A8020844A80208FF00420039
:10476000F8B50400012803D92A492B48FFF7E2FDD8
:10477000FFF786FE85B2FFF78CFE0700002080263B
:10478000FEF79CF87600002811D1B74211D1222DF6
:104790000FD88025214B6D041B6824065968204BD7
:1047A0002C40CA581F4D2A401443CC50F8BDB74284
:1047B00029D0FFF75FFF0500B7420FD1621E944179
:1047C000802362425B001A40174BD2180121280057
:1047D000FDF7AEFD002808D01448E7E7621E9441BB
:1047E000022362421A40124BEFE70C4B1B68B433B2
:1047F0001B68EB181A68002AFCDBEB6800201B0E14
:10480000A02BE9D1D2E7222DE6D9FFF733FF05002F
:10481000D4E7C0467F0A00003B840D10E0AD0208DB
:1048200018F00000FFFFFFFE01000030040042000E
:104830000100000CF7B50700012803D929492A48CF
:10484000FFF778FDFFF725FE80235B0098421CD020
:10485000FDF75FFAB0230190244D254A5B05002F38
:104860001AD0244903205958A950234A23499C5C53
:104870001F226B58E4B293431A000B2313436B506F
:10488000FFF74EFDFFF7B2FE12E0FFF7E3FE002850
:10489000DED11B4E3000FEBDAF50E8220120D20019
:1048A0009C5CFFF75DFFE4B2061E0DD1FFF7FCFD37
:1048B0001F21124A0C40AB588B431C43AC50002FB5
:1048C00006D1FFF765FE3E000198FDF726FAE1E705
:1048D0000720FFF725FDFFF723FE0020FFF740FF2D
:1048E0000600F1E7530800003B840D10000026404D
:1048F000307F000010180000410700001CFF00007E
:104900000300420010B5041E03D111491148FFF7FE
:1049100011FDF222104BD2011B68DB689A5822600D
:10492000F022D2019A5862600C4A9A58A2600C4A4E
:104930009A58E2600B4A9A5822610B4A9A5862616F
:104940000A4A9A58A2610A4A9B58E36110BDC046C0
:10495000D40A00003B840D10E0AD0208047800008A
:10496000087800000C78000010780000147800002F
:104970001878000010B5041E03D110491048FFF745
:10498000D9FCF0220F4B61681B68D201DB6899509B
:10499000A1680D4A9950E1680C4A995021690C4A66
:1049A000995061690B4A9950A1690B4A9950E16984
:1049B0000A4A99502168E832995010BDFC0A00005B
:1049C0003B840D10E0AD0208047800000878000078
:1049D0000C780000107800001478000018780000AF
:1049E000F7B50700012803D940494148FFF7A2FC69
:1049F000404D6B68002B4AD1FDF78BF96B68019035
:104A0000002B56D13C4E33681A0043321278002AEC
:104A100007D09B68E0331B68DB0602D53748FFF7F9
:104A200071FFFFF736FD80235B00984246D13800C6
:104A300003F05AF8002433681A0043321278002A2F
:104A400017D0002815D09B68E0331B68DB0610D513
:104A5000FFF716FD294B212808D032681300B03328
:104A6000198807234B43126A9B18DB681800FFF76D
:104A700081FF0198FDF751F9002C0ED16B68002BD6
:104A800003D008210120FFF709FE2000FEBD01210F
:104A90000800FFF703FE041EAED06B68002B03D0A6
:104AA00002210120FFF7FAFD154B9C42EDD0154C79
:104AB000EBE704210120FFF7F1FDA3E7FFF7DAFDA3
:104AC0003368B4331B68C0180368002B0BDB042366
:104AD0000D4A11690B431361012F02D030BF002032
:104AE000A8E720BFFBE70020054CA4E7AE020000CA
:104AF0003B840D1048A80208E0AD020824A8020873
:104B000005004200FF00420000ED00E0C0228020CE
:104B1000064952008B58C0059B009B0803438B50ED
:104B2000802388581B0603438B50704700002640A3
:104B30007047FFF7FDFF72B6124C134DAC4209DA15
:104B400021686268A368043B02DBC858D050FAE7CA
:104B50000C34F3E70D4B0E4CA34208DA19685A687F
:104B60000020043A01DB8850FBE70833F4E70948EA
:104B700009490860BFF34F8F00F0E4F800F09CFA99
:104B8000FEE700005C8C0D10748C0D10748C0D1001
:104B9000848C0D1000A0020808ED00E0FEE7FEE79F
:104BA00000B504207146084202D0EFF3098001E00D
:104BB000EFF308800430FFF7EDFBFEE770470000DD
:104BC000E02370B5504C9B00E2580F23D021072002
:104BD00013409A00121989005158014066D00429E7
:104BE00058D04A48002B66D1B223B1220321DB0002
:104BF000D200E558A358A6581B0F360F0B400E42A3
:104C000004D0A258120F0A40012A01D1EA0701D4A8
:104C1000032B11D1B0233E4ADB00E558A158E658DA
:104C2000C904C90C02F064FBAD03AD0B6843F1018C
:104C3000C90F013102F05CFBE0239B00E3589B06A7
:104C40009B0FD840334B1860334B1C691969240AF9
:104C5000090E013102F04CFB304BE1B2186001311A
:104C600002F046FB2E4B040018602E4B2E491860B4
:104C70002E4BC01802F03CFBFA212D4B8900187016
:104C80002C4BE01802F034FB2B4B18602B4BC0036D
:104C9000186070BDC021890052581F210A40112A96
:104CA00001D0132A04D1802000029BE7244899E711
:104CB000FA20C00196E7012BBED1C823C0220321F0
:104CC000DB00D200E558A358A6581B0F360F0B4047
:104CD0000E4204D0A258120F0A40012A01D1EA075D
:104CE00001D4032BA8D1C022D200A358A158A558A3
:104CF0007F221F261340090A3140584302F0F8FA78
:104D0000290C314096E7C0460000264000366E016F
:104D10008405000020A102080000214024A102080F
:104D20001CA102082CA1020840420F003F420F00C4
:104D300034A10208E703000030A1020828A10208FC
:104D400000127A0010B51B48FCF7EAFFB022E02100
:104D50003020194CD200A35889005B005B08A35097
:104D600063588343635080235B04A350134B144A5E
:104D7000E250A02204339201E250FF22114BE25094
:104D8000FFF7C4FEC02201215200A3588B43A35059
:104D9000FFF714FFFFF714FFB0235B055A78002AD2
:104DA00002D05B78212B03D10022074BDA605A60D6
:104DB00010BDC046F47F0D100000264084050000A1
:104DC000010002008C050000E0002340024BD86F78
:104DD000032318407047C0460400214010B5FCF77B
:104DE00098FF0749074ACB6F1A40074B1343CB671D
:104DF000102306490A681A42FCD0FCF78EFF10BD4A
:104E000004002140FCFF00000100FA058800214059
:104E100070B583050600002B04D0E8211048FF314F
:104E2000FFF788FA0F4CFCF774FFE36F0500DB43D4
:104E30009B0701D1FFF7D2FFB0230B4A9B00D6504E
:104E4000E36F0A4A0A491A400A4B1343E3671023E7
:104E50000A681A42FCD02800FCF75FFF70BDC0460C
:104E600093840D100400214000002140FCFF00004D
:104E7000880021400300FA0510B562B600F0BCF9C5
:104E8000FFF744FEC0220120024952008B588343A1
:104E90008B5010BD0000264010B50020FDF71EFC11
:104EA00010BD0000802310B50C4C032023602300AC
:104EB000210008336360FDF741FC0948FDF76CFAF7
:104EC000084B1B6851331B78002B02D00648FDF7B6
:104ED000DBFA20001830FCF7D3FF10BD00C0020839
:104EE0003CC00208E0AD020800850D1010B5044872
:104EF000044A0021121A02F005FCFBF7F5FA10BD76
:104F00000000020800A002080022E82313B5019265
:104F1000019C9B0523430193019B090419430191C3
:104F2000019B000218430123019001990B43019357
:104F30000199124BD96012491868002806DB8A4291
:104F400002D10120404216BD0132F5E78A42F8D075
:104F500001229A6000221869002803DA8A42F0D000
:104F60000132F8E78A42ECD0DB6800200193A023ED
:104F7000019A1B069A42E6D00198E4E7000023401C
:104F8000983A000010B5084B0024DB78013B012B58
:104F900007D801210800FFF7B7FF04006420FFF7DE
:104FA000A5F9200010BDC0463CAF0208A02270B594
:104FB0000E4DD200AA580400032A01D0FFF7E2FFE9
:104FC0000B4B1B68002B06DA0A4B0B4ADA6472B6ED
:104FD00002F0A2FD62B6AC239B00EC50074B9C6034
:104FE000236883F3088863689847FEE70000214040
:104FF00000012640000023402143341200ED00E070
:1050000070B50400FFF7BEFF144B1B68002B1DDAC0
:10501000134B144ADA6472B6B023134A134D9B0043
:105020001348EA50C36F134A13491A40134B1343F2
:10503000C36710230A681A42FCD00120FFF756F913
:10504000B0239B00EC5002F067FD62B62000FFF732
:10505000DFFE0020FFF7C4FCFBE7C046000126404E
:10506000000023402143341200400016000021407C
:1050700004002140FCFF0000880021400300FA05E5
:1050800010B500280ED1FFF77DFF074B1B68002BE2
:1050900003DA064B064ADA6472B60648FFF7B8FE32
:1050A00002F02AFD10BDC04600012640000023404A
:1050B000214334120040001670B586B0FFF7F2FEAF
:1050C000FFF7DAFE8020424A424B01A91A604000F5
:1050D0006A46FCF743FD041E34D13F4D03003F4AAE
:1050E00029000198FBF7BEFB041E2BD1AB78022BE5
:1050F00000D9A870F022EB68394E12069B18B360F5
:105100002B69F3606B699B18F361AB693362FBF742
:10511000B7F9041E16D1AB78002B1ED0314A013BE3
:105120009B00314D9B582B6000F0D2FB2F4A0600AC
:1051300029682F4800F024FC002E14D101212C48AE
:10514000FEF742F86042604103ACFFF799FF200090
:1051500001F066FC002808D0FEE7264BF2699A426F
:10516000F0D96C70EEE73400ECE702A9207900F08A
:1051700094FC43425841FFF783FF029BA468E41864
:10518000039B1B89E418FFF7B1FE43425841FFF728
:1051900077FF114B1878042818D802F09FF8030302
:1051A00007070F002000FFF701FFFEE702210020A4
:1051B000FDF752FB2000FFF7F9FEF6E706210E206F
:1051C000FDF74AFB2000FFF71BFFEEE7FEE7C046B6
:1051D0004C850D10E4AD0208E8AD02083CAF0208B2
:1051E00040A1020838A102085CA80208CCAF02085E
:1051F00000004240FFFFFF0710B500F009F800F083
:1052000035F800F043F800F005F900F02DF810BD76
:1052100080218022124BC9001B68D205986810B506
:1052200042501A00743212880E4C12181068044052
:10523000D4208001204310601C001A0072347032A8
:105240002478127898687333A2401C780323A34013
:1052500013438022120613434350435810BDC046E7
:10526000E0AD0208FF00FFFF70470000054B1B6820
:105270001A003F321278052A03D900219A68024B9E
:10528000D1507047E0AD0208140C000010B51D4C61
:105290001D4A00212000FCF7CDFE20001B4C1C4ABB
:1052A0000121FCF7C7FE1B4A02212000FCF7C2FEC9
:1052B000194A03212000FCF7BDFE184A04212000F2
:1052C000FCF7B8FE164A05212000FCF7B3FE154A8C
:1052D00006212000FCF7AEFE2000134C134A0721E4
:1052E000FCF7A8FE124A04212000FCF7A3FE114A95
:1052F00006212000FCF79EFE0F4A07212000FCF744
:1053000099FE10BD00003240A0860D10800532408D
:10531000D4860D106C860D1004860D10D0850D10EE
:105320009C850D1068850D100003324038860D10E5
:1053300008870D103C870D1070870D1010B50A4BB3
:105340001B683E331B7883420BD9E0220F24074BA6
:105350008000C01892008358A34319438150002055
:1053600010BD0348FCE7C046E0AD0208000026403F
:1053700001004A0010B50A4B1B683E331B7883427C
:105380000CD9E0223024074B8000C01892008358CB
:105390000901A34319438150002010BD0248FCE7D6
:1053A000E0AD02080000264001004A00054B064916
:1053B0001B681A000832D26F1B689B181A680A40D3
:1053C0001A607047E0AD0208FF00FFFF074B1B6843
:1053D000190008311A68CB6F8021D218136849046C
:1053E0001B021B0A0B4313607047C046E0AD020866
:1053F000054B06491B681A00883212681B689B1807
:105400001A680A401A607047E0AD0208FF00FFFF0B
:10541000FEE70000F8B596210020FEF7D3FFFEF767
:10542000A9FF002801D1FEF793FF0120FFF702FA40
:10543000644B65495A6C0A40E82189010A435A6461
:105440005A6C120AD2B23A2A04D15A6C5F4802400E
:105450001143596400210800FFF78CFFFFF7C8FFD4
:10546000FFF7B4FFFFF7A2FF594D5A4C2B685A4F74
:105470003D331B78002B0ED0C0268023F600A259A6
:105480009B053A401343A3510120FEF749FFA3595E
:105490005B005B08A35100210120FEF705FD2B688E
:1054A0003E331B78002B03D14C494D48FEF742FF99
:1054B000E0239B00E6580F231E400AD13000FEF780
:1054C0001BFD1223FF33984203D101213000FFF767
:1054D00035FFB122D200A35800213B408027BF05F1
:1054E0001F43A750083AA35808005B005B08A3506D
:1054F0003C4AA3585B005B08A350FEF7D5FC002193
:105500000800FFF71BFFFFF773FFFFF75FFFFFF7D1
:105510004DFF00210120FEF7C7FC01210020FFF70D
:105520000DFF00210800FEF7BFFC00210220FEF75E
:10553000BBFC00210320FEF7B7FC00210420FEF78E
:10554000B3FC2948FEF7FEFC002802D00420FFF738
:105550005FFF2648FEF7AAFD002802D00420FFF7CF
:1055600057FF00210800FFF7E9FE00210800FFF7C0
:1055700001FF00210120FEF797FC00210220FFF728
:10558000DDFE01210220FFF7F5FE2B683E331B787C
:10559000022B06D9E22280239200A1581B060B435E
:1055A000A3508022124B1206E15800200A43012129
:1055B000E250E2580A43E2506331FEF703FFFFF77F
:1055C000FFFAF8BD00002740FF00FFFFFFC5FFDF27
:1055D000E0AD020800002640FFFFFFCF6E0600008E
:1055E000A4870D108C05000000880D10400D0300ED
:1055F0000C050000437802781B021A438378C078B8
:105600001B0413430006184370470000F7B5A54B71
:10561000A54A9A58D10700D47BE00F22A34FBB685C
:105620003D680093A24BDC6F0193009B1440073A46
:10563000141B9C4200D91C009E4E002C18D1009BCC
:105640003D60BB60002B0CD1F92201209549D200AE
:105650008B5883438B50B861FB69002B01D0FB69E9
:105660009847F8230122DB008E49CA50CB58F7BD7A
:10567000082C16D12800FFF7BDFF3060281DFFF76A
:10568000B9FF3060009B2D191B1B0093019BDC6F41
:105690000F231C40073B1C1B009B9C42CDD91C00C8
:1056A000CBE7012C03D12A78834B1A60EAE7022C5E
:1056B00006D12A786B781B021343804A1360E1E716
:1056C000032C07D16B782A781B0213437B4A1360A3
:1056D000AA78E9E72800FFF78DFF042CD1D03060CD
:1056E000052C01D12A79DFE7062C02D12A796B79C2
:1056F000E1E7072C07D16B792A791B0213436F4A24
:105700001360AA79D0E7281DFFF774FF08243060E2
:10571000B8E7910700D4A4E00F22644D68496C6992
:10572000EB6808688C460240A24200D92200654915
:10573000654E002A16D1EB606C61002C0DD1F92268
:1057400002215848D20083588B4383500320A8611C
:105750002B6A002B01D02B6A9847F8236C61DB0081
:10576000022281E7082A19D10868070A18705F70B9
:10577000070C000E9F70D8700868070A18715F71D7
:10578000070C000E9F71D8719B18A41A62460F2057
:1057900012680240A242CCD92200CAE7012A03D1F2
:1057A0004A4800681870EFE7022A04D13068187080
:1057B000000A5870E8E7032A07D130681870000A19
:1057C0005870424800689870DEE7042A08D10868DB
:1057D000070A18705F70070C000E9F70D870D3E72F
:1057E000052A0BD10868070A18705F70070C000EB5
:1057F000D87036489F7000681871C5E7062A0CD12A
:105800000868070A18705F70070C000E9F70D87048
:1058100030681871000A5871B6E7072A0FD1086876
:10582000070A18705F70070C000E9F70D870306800
:105830001871000A5871254800689871A4E70A6831
:10584000100A1A705870100C120E9870DA700A68EC
:10585000100A1A715871100C120EDA719871082220
:1058600092E704210A4207D00520104A9061F822ED
:10587000D20099509B58FAE608210A4202D00B4AFE
:105880000620F3E71020024206D00721074A916163
:10589000F822D2009850EDE72020024200D1E6E63F
:1058A000024AF4E700004240CC070000CCAF0208F7
:1058B000080042409800424090004240940042401C
:1058C000C4004240D8004240D4004240D000424090
:1058D00037B568460200154B12CB12C262B61449A6
:1058E000FEF7B0FCFA22134D92002B001249134828
:1058F000FDF71CFC041E13D1020001210F48FDF727
:1059000079FC29000D48FDF79FFE2A000C490B4841
:10591000FEF79AF9041E03D101000848FDF754FC74
:105920008022084B20001A603EBDC046A48A0D109C
:105930000D560D10CCAF020858850D1000004240E6
:10594000948A0D1000E100E00C4B1B689B691B68FA
:10595000032B08D10023CB7083B21B0A88704B70D5
:10596000000C08707047042BFCD183B2C8701B0A6E
:10597000000C48708B70000AF3E7C0465CA8020870
:10598000F0B50F2787B002ABFF18002316003B705D
:105990008B690500DA6BDB6A03921B683A00DBB2A5
:1059A00000960C00FDF77AFE002813D16B463A787A
:1059B0001B7B1A409A420DD0320021002800FDF7CF
:1059C000C7FE002806D1320021002800FDF784FE22
:1059D0000028F8D107B0F0BDF0B589B004000E0082
:1059E000049217221A4D0593296802A88B69121890
:1059F0009F6ADB6A20001B680096DBB2FDF74EFE53
:105A0000002823D1320029682000FDF72BFE002852
:105A10001CD1059B019000930296049B0E9A296865
:105A20002000FDF709FF002810D13200296820006E
:105A3000FDF752FE0028F8D117223B6802A9009614
:105A40005218DBB229682000FDF728FE09B0F0BD2E
:105A50005CA8020870B54B68056801229D4216D308
:105A60008A689B1800229D4211D20C694B699C42A6
:105A70000FD20C236343CE680134F3180E685A70BA
:105A80001E705A8042685D609A6001220C611000AD
:105A900070BD0C235B428B61F9E76F2804D1802332
:105AA00000205B050B60704716204042FBE70000BA
:105AB00010B50F4B02001879904215D0187E904215
:105AC00014D018002C3004780120404294420AD1AE
:105AD000033014224243101D1818086000209B1840
:105AE0001A6901321A6110BD0020F2E70120F0E7C7
:105AF00040A10208002809D00438054B02689A42E8
:105B000004D10369002B01D0013B03617047C046FB
:105B1000EFBE0DD070B544680C480C19012115007A
:105B20001E00FDF751FB80235B05E218084B9A42EB
:105B300003D9084B9B78002B05D0320029002000A8
:105B400000F030F970BD01204042FBE70000424008
:105B5000FFFFFF17E8AD0208F0B51500F0221A4F5D
:105B600087B003933B684468DB6812060C199B18E6
:105B7000A34216D800211548FDF726FB3B6805AE69
:105B8000D8688023201A5B05C0183100FFF7DCFEBF
:105B90000096039B2A000E490C48FFF71DFF07B033
:105BA000F0BD80230B4A5B05E318934203D90A4BEF
:105BB0009B78002B05D0039A2900200000F088F97B
:105BC000EDE701204042EAE75CA8020800004240FD
:105BD000CCAF0208FFFFFF17E8AD0208F0B51500D3
:105BE000F0222B4F44683B681206DB680C199B18A7
:105BF000C5B0A3423AD800212648FDF7E5FA802235
:105C00000021520004A801F07DFD3B680020D96806
:105C10008023641A5B052E0AE418002E14D0002895
:105C200001D045B0F0BD03AF20003900FFF78CFE76
:105C3000802300975B0004AA174916480134FFF738
:105C4000CBFEFF34013EE8E7EDB2002DE9D000289D
:105C5000E7D103AE31002000FFF776FE00962B005F
:105C600004AA0D490B48FFF7B7FEDAE780230B4A79
:105C70005B05E318934203D9094B9B78002B04D0B2
:105C80002900200000F02EF9CBE701204042C8E7B0
:105C90005CA8020800004240CCAF0208FFFFFF17DB
:105CA000E8AD020810B5007800F08CF910BD0130A5
:105CB00070470000431E022B15D8022808D0032885
:105CC0000BD00A4B98680860DB68002013607047AF
:105CD000064BD86908601B6AF7E7F0231B030B60CB
:105CE00080235B01F1E701204042F0E740A1020878
:105CF00030B589B00C00150002A903AA0190FFF786
:105D0000D9FF002811D1236805900693084B07900E
:105D100001AA18680749049500F00EF807980028B2
:105D200001D1059B236009B030BD01204042FAE754
:105D3000E4AD0208555A0D10F0B500242600436862
:105D40008BB002911B6906A905A80392984701949C
:105D5000069BB34201D80BB0F0BD059BF700DF19DD
:105D60007B68019D0893019B3A68EB1A9A4202D81E
:105D700001360195ECE707940995039907A8029B62
:105D800098470028E7D0089B0135E418EBE70000AE
:105D9000024B036001230B607047C046AC8A0D10B4
:105DA000002070470B00802110B5490541181800EC
:105DB00001F09FFC002010BDF0B5264CF023A54457
:105DC0000024039020001B06CB1801935B0A5B02A2
:105DD00004AF0292FD1A029AA24201D900280CD007
:105DE0001D4B984234D01D4B984231D0431E9841F0
:105DF000400085239B009D44F0BD8022010092005D
:105E00009E18019A9A421DD8029AA2421AD9039A60
:105E1000125DEA54002906D18021490559180978F4
:105E2000511A4A1E914101340133B342E9D100298C
:105E300004D00B4B3900F018FCF782F8094BED1831
:105E40003300C8E7802252059A181278EA54EBE72B
:105E50000120CEE7ECFDFFFF0200520006005200D9
:105E600000FEFF0F00FEFFFF00207047F8B5124C48
:105E70000023A1421CD91E00104C8D18AC425E417B
:105E80000F4CA14215D91F000E4CAC425F413C00A3
:105E90000D4FB94202D90D4FAF425B41344323430A
:105EA0000124002B02D0FFF787FF04002000F8BD7B
:105EB0001E0000242300F1E7FFFFFF0F0000101079
:105EC000FFFFFF1300800014FF070016000A0016F2
:105ED0000B00802110B5490541181800FFF7C6FFD7
:105EE00010BD00008023F0B55B05C0184518334C89
:105EF000EB05A544C605DB0DF60D01936B0A039374
:105F000033005A1E9341400AC0186B0A1B1A0093B3
:105F100043021F0000240293009B002B3ED1002E61
:105F20001AD0274A029B944663441C001900320091
:105F300004A801F0DEFB2000FBF7C4FF43425841F8
:105F4000FFF79EF82100320004A8FFF78FFF04003E
:105F500060426041FFF794F8019B002B19D0802428
:105F6000A400E41A2200290004A801F0C2FB039B4C
:105F70005802FBF7A7FF43425841FFF781F8220080
:105F8000290004A8FFF772FF040060426041FFF798
:105F900077F8200085239B009D44F0BD3800FBF777
:105FA00091FF040060426041FFF76AF880239B0084
:105FB000FF18009B013B0093AEE7C046ECFDFFFFDE
:105FC00000FEFFFF0420704710B5102209490400AD
:105FD00001F080FB0123002808D023001033226841
:105FE000013205D104349C42F9D10323180010BDBD
:105FF0000223FBE7CC8A0D1030B5040091B00120DC
:106000000D00FFF73DF8A168102310396A46200003
:10601000FFF780FD002802D0012011B030BD684696
:10602000FFF7D2FF28702378032B0CD10120FFF754
:1060300027F8A1680123AA1C18392000FFF76AFD80
:10604000431E9841E9E70120FFF71AF80120FFF706
:1060500017F8A1686A1C203901232000FFF75AFDB8
:106060000028E3D0D8E737B50D00C0B201A9FFF78B
:106070001FFD0124002807D129000198FFF7BCFF6C
:1060800004000198FFF736FD20003EBDF7B5012062
:106090006946FFF7E8FF002838D101AC2100023043
:1060A000FFF7E1FF002831D12078A678184C6B4625
:1060B000220019789D785F7812322378002B01D066
:1060C0008B421ED16378002B01D0834219D1A37873
:1060D000002B01D0AB4214D1E378002B01D0B342A6
:1060E0000FD12379002B0AD1022200206379023BD1
:1060F000DBB29A424041FEF7C3FF6079FEBDBB426E
:10610000F2D006349442D8D10120F7E7FF20F5E71A
:10611000DC8A0D10F0B597B01CAB1B78039004938C
:1061200013781400302B16D19378022B13D106ADBF
:1061300040220021280001F0E5FAE278A1184B790D
:10614000901D0979C0180290022904D1D1186078F5
:10615000043188422AD0102017B0F0BD059A0F1ADA
:106160005618B446A444664636790822B44604AEAE
:10617000B61862462037F25501318842EED100222E
:106180000299C91A64189A420AD16B46188A4023A8
:1061900000950193039A203B0A49FAF7D9F9DBE706
:1061A000D11AA05C403168540132ECE7202B00DDAD
:1061B00020231000202A00DD2020121A0021059241
:1061C000DBE7C04609000610002803D1044B1B7F03
:1061D0001800704700230128FAD1014BDB7FF7E755
:1061E000E8AD0208F0B5F7B00500029111A85949D1
:1061F00017000493FAF734FA00284CD17C9B002B4B
:106200003FD100242B89EA689B180393039BA34288
:1062100014D9039B049E1B1B9E4200D91E00330011
:106220003A0021000298FFF775FC002833D13200B4
:10623000390011A8FAF722FA00282ED008AB202244
:1062400009A911A8FAF72AFA002824D17E9B002B6D
:1062500004D0202209A9180001F04BFAEB682C8920
:1062600007ADE4182A00042321000298FFF752FC2E
:10627000002810D1384B2A889A4210D00120404281
:1062800009E07D9B002BBCDD1A007C9911A8FAF770
:10629000F5F90028B5D077B0F0BDA419B6E76B8842
:1062A00001251B1905930434039004906D42059B4E
:1062B0009C4205D3049B002BE0D003980138EAE709
:1062C00008AF04233A0021000298FFF723FC0028BE
:1062D000E1D13B787E88102B17D1202ECED1211D05
:1062E000330011AA0298FFF715FC0028D3D1320021
:1062F00011A909A801F0EEF90028BFD101230493E8
:1063000008AB5B880433E418D1E7012B04D17F98F4
:10631000FFF75AFF0500F3E7222BF1D13300483B8A
:10632000B82BABD8211D330011AA0298FFF7F2FB5E
:106330000028A3D1EDB27B8811AA0095202109A8DD
:106340000125FFF7E7FE6D420028D9D10123039311
:10635000D6E7C0460900000107690000F7B507004D
:10636000002401262000FFF7A2FC01A9C0B2FFF71C
:106370009FFB3500011E0AD12C2363430B4A019871
:10638000D2182023FFF7C6FB0500681E854101983F
:10639000FFF7B0FB002D04D0012C00D13D002800F8
:1063A000FEBD012CFBD03400DCE7C04660A802082B
:1063B00073B50C00C0B201A91500FFF779FB0126E7
:1063C000002807D12A0021000198FFF707FC0600EA
:1063D000701E86410198FFF78DFB300076BD0000EE
:1063E000F0B52C244443304B87B01C1923680500BA
:1063F0001A002E4B9A4201D001204AE02369DB06A5
:10640000FAD4FFF754FC04A9C0B2FFF751FB030014
:106410000120002B3ED1E368268905AFF6183A002B
:10642000042331000498FFF775FB0028E4D1204BCA
:106430003A889A4201D1788880192C236B431A4AF2
:10644000D3181B6A9B688342D6D31A4BA27A1B7857
:106450009A42D1D12000F9F795FE0028CCD12368CB
:106460001A00124B9A4217D180230290019000909B
:1064700003955B00104A04992000FFF7B3FE002843
:106480000AD10498FFF736FB2000F9F79FFE431E60
:106490009841404207B0F0BD002DADD004980021D6
:1064A0008268FFF79BFBA7E760A802083DB8F39658
:1064B00007690000E8AD0208D0AC02080023F0B57F
:1064C000B04CB14AB14DA544012013602B60FFF7D9
:1064D00087FFAF4B040001201F79FFF775FE002CEA
:1064E00047D1AC4BC2B2DB6C39005E6880235B05E0
:1064F000F3180293A84BF618300013ABFBF766FBBA
:10650000041E36D105A8FAF7EDF88021A34A8900C8
:1065100005A8FAF7F5F805A90B20FAF701F9041E0A
:1065200027D1102313AA9E490B20FAF7C9F801239B
:10653000041E2B601DD1994A0B211BA8FAF71CF8E9
:10654000041E16D1102217A91BA8FAF737F8041E4B
:106550000FD1202204AB2DAD019300922B0031000E
:106560001BA8FAF73BF8049B0400202B10D0012451
:106570006442864B1B68002B05D00B20FAF744F8C9
:10658000002800D004002000D3239B009D44F0BDD0
:106590000028EED1020004AB29001BA8F9F7FCFF8C
:1065A000041EE6D107AE33002A0013CA13C37D4F81
:1065B000126831A91A603800102201F09AF805A972
:1065C0000C20FAF7ADF8041ED3D110233200744921
:1065D0000C20FAF775F801226B4B041E1A60C8D123
:1065E00071496DA8FAF73CF8041EC2D1029B029AC9
:1065F0001B890C21D3181BA8684A0393F9F7BCFF29
:10660000041EB6D1102239001BA8F9F7D7FF041ECB
:10661000AFD1802604AB7600019300962B003200A8
:1066200003991BA8F9F7DAFF049B0400B3429ED13B
:1066300000289ED12D9B2E89AA7A309F3199581C13
:1066400000D194E7C90600D591E75249C96C896821
:10665000B94200D28BE755498B4200D087E74C4BBB
:106660001B78934200D082E78022290052006DA857
:10667000FAF704F8041E00D07BE7F619330AF6B2E5
:10668000771EBE4101279B190293039B3E029E1970
:10669000029BBB4222D9002C00D06AE704AB0193D5
:1066A00080232DAA5B00009313008022310052004A
:1066B0001BA8F9F793FF8023049A04005B009A4219
:1066C00009D1002805D11A002DA96DA8F9F7D6FF28
:1066D00004000137D9E701246442FAE7002C00D016
:1066E00047E704AF3B0020220BA96DA8F9F7D6FFBE
:1066F000041E00D03DE780225200019700922B003B
:1067000031001BA8F9F76AFF041E00D031E7020030
:106710003B0029001BA8F9F73FFF2D9B244A9BB2A1
:106720000400934200D022E7002800D021E72E9AEF
:10673000D3B2102B00D01AE7120C202A00D016E793
:106740002FA90BA800F0C6FF041E00D011E7379B4D
:10675000DBB2012B00D00AE70120FFF735FD409B9B
:10676000DAB2222A00D002E71B0C482B00D0FEE64A
:10677000C0B2009041AA20210BA8FFF7CBFC040077
:10678000F7E6C046B4FCFFFFFCAF0208F8AF020812
:10679000E8AD020860A802082000001000016004B3
:1067A00001000040C0AC0208090000013DB8F396AA
:1067B000076900000023F0B51D4C0700A544694699
:1067C000022000930193FFF773F900280ED00126F1
:1067D0000098002801D0FFF78DF90198002801D01A
:1067E000FFF788F93000134B9D44F0BD01A901204B
:1067F000FFF75EF90600041EE9D10098A742E7D929
:1068000080233D1BDB009D4200D91D002B0002AA06
:106810002100FFF77FF90028D9D12B0002AA21001F
:106820000198FFF799F90028D1D16419E5E7C0462E
:10683000F4FBFFFF0C040000F0B500242500584FC6
:106840009BB0BB6A0293029BAB4263D1554BDB7892
:10685000002B00D19FE0002305A902200593069399
:10686000FFF726F9002821D106A90130FFF720F90A
:1068700000281BD14C4A0C2108A8F9F77DFE0028FE
:1068800014D11022494908A8F9F798FE041E0DD129
:106890000600BB6B0133FF330293059B5B680393D8
:1068A000029BB34200D86CE0002C44D0059800282D
:1068B00001D0FFF71FF90698002801D0FFF71AF959
:1068C0003B4B1B68002B02D00C20F9F79DFE1022D9
:1068D0000021364800F016FF3B6D00219A68022027
:1068E000FFF766FD43425841FEF7CAFB0C237A6D61
:1068F000396D013A5343CB185A6849680220511A3E
:106900009A68FFF755FD43425841FEF7B9FB002056
:106910001BB0F0BD0C236B437A6A2100D3189E682C
:1069200001203200FFF744FD43425841FEF7A8FB27
:10693000A419013587E7029B9D1B8023DB009D4244
:1069400000D91D00039B009599191A4B2A00C918FC
:1069500007AB019308A8184BF9F740FE079B04000A
:10696000AB420BD100289BD12B00134A3100069873
:10697000FFF7F2F8002899D1761991E701246442D3
:106980008EE7002C00D091E707AB22000A4908A847
:10699000F9F702FE8AE72000FFF70CFF9CE7C046EC
:1069A00060A80208E8AD020800016004C0AC02085B
:1069B000FCAF020800040010C0A8020873B5164E10
:1069C000164CF368626A5B0A01A901200193FFF784
:1069D0008FF9012500281AD1019B226DA362F3686B
:1069E00001A95B0A02300193FFF782F9051E10D15D
:1069F000019B206A6365FFF755F90600A06DFFF75C
:106A000051F9331C864200D2031C5C3423702800E9
:106A100076BD0125FBE7C04640A1020860A8020838
:106A2000F0B50C265A4F89B0FB6800905C0A74439D
:106A3000200000F029FE0190200000F025FE019BBF
:106A4000544C0290636220650020FFF730F921006A
:106A5000C0B22031FFF72CF843425841FEF710FB3B
:106A60000120FFF724F92100C0B24C31FFF720F8D4
:106A700043425841FEF704FB210003205831FFF741
:106A800017F843425841FEF7FBFAFFF797FF051E40
:106A90006BD1FFF763FC051E67D1FB68A06A5B0A38
:106AA00098424FD8626D9A424CD890424AD10823FE
:106AB0004643626A216D08369E4226D1364E73786F
:106AC000002B3FD00C22002105A800F01BFE012066
:106AD000FEF7D6FAFFF7DAFA831E0500022B07D875
:106AE000F378002B19D0FFF7E9FC00281BD005250F
:106AF0000120FEF7C5FA012D24D0002D01DD052D62
:106B00001BDD0020FEF7BCFAFEE71800D558CB5875
:106B10000C309D4216D10300CEE70120FFF760FC48
:106B2000E3E7032521E00120FEF7AAFAFFF784FE40
:106B300043425841FEF7A4FADAE70020FFF70EFCC3
:106B4000051E12D10020FFF74BFC0500684268418A
:106B5000FEF796FA002DE4D1236A00995A780A715B
:106B60005B680C600393039A8A60019800F096FDBD
:106B7000029800F093FDA06DFEF7BCFFE06CFEF7FD
:106B8000B9FF206AFEF7B6FF280009B0F0BDC04685
:106B900040A1020860A80208E8AD020810B501781B
:106BA00004000A00303AD3B2092B1FD811000A01A1
:106BB00061780B00303BD8B2092824D89918A27804
:106BC00009011300303BD8B209282AD85A18E378B3
:106BD000120118003038C1B28018092905D91900EE
:106BE000413905292BD8373B981810BD0B00413B84
:106BF000052B01D83739DAE70B00613B0020052B64
:106C0000F3D85739D3E70B00413B052B02D837396E
:106C10008918D4E70B00613B0020052BE5D85739D4
:106C2000F6E71300413B052B02D8373A5218CEE75E
:106C30001300613B0020052BD7D8573AF6E719001F
:106C4000613900200529D0D8573BCDE7F7B50B783F
:106C500007004E1C222B0FD00026554B1960300028
:106C6000FEBD02331A780130222A08D0002A06D04D
:106C70005C2AF6D00133F5E733000020F2E74D4BF4
:106C80001B6898470190041E07D1019EE7E7721C1C
:106C90005C2B13D02370013416003378222B01D0E3
:106CA000002BF4D1002323703378223B5A42534106
:106CB000F618019B3B610423FB60D0E773786E2BD1
:106CC00017D007D8611C622B0CD0662B0FD0237015
:106CD00001340AE0742B0ED0752B0ED0722BF6D136
:106CE0000D23F4E7082323700C000132D4E70C23B2
:106CF000F9E70A23EBE70923E9E7B01CFFF74EFFAA
:106D00002D4B2E49C3180500721D8B42EDD900286A
:106D1000EBD02B4BC3188B4227D8B3795C2BE4D133
:106D2000F379752BE1D130000830FFF737FF3200DF
:106D3000214B2249C3180B328B42D6D8214BAD02CE
:106D40001D4080238005800D05435B02ED181E4B1E
:106D5000E11C9D4223D803234C1E3F208021284064
:106D6000494201432170AD0910E07F2809D8012371
:106D700001341648611EC05C013B05430D70E418E8
:106D8000B3E7134B9842E2D8022302343F2080211C
:106D900028404942013C01432170AD09E9E73F2009
:106DA000802328405B420343E370AD090423D3E70B
:106DB000D0AD020880A102080024FFFFFF030000FD
:106DC0000028FFFF00FC0F00FFFF0000EE8A0D10FF
:106DD000FF070000002803D00378013B1F2B00D9D8
:106DE00070470130F6E70000064B10B51B682820FD
:106DF0009847041E03D02822002100F083FC2000C5
:106E000010BDC04680A10208F0B5050087B00E1E77
:106E100001D1002413E004227549300000F054FD34
:106E2000002803D10223EB60341D08E005227149DC
:106E3000300000F049FD002804D1E860741D2000F6
:106E400007B0F0BD04226C49300000F03DFD002881
:106E500006D101230122EB600023AA61EB61E3E785
:106E60003378222B05D131002800FFF7EFFE040014
:106E7000E5E71A00303AD2B22D2B01D0092A1AD8F0
:106E8000340000E0013423781A00303A092AF9D995
:106E90002D2BF7D0A71B3A003100684600F029FCE3
:106EA00000236A466846D35500F0E4FB0323A8613B
:106EB000E961EB60C3E75B2B37D1563BEB60701C9D
:106EC000FFF788FF037804005D2B01D10134B6E79A
:106ED000FFF78AFF061EA8609BD02000FFF77AFF0D
:106EE00001003000FFF790FFFFF774FF0400002C53
:106EF00000D18EE723782C2B04D05D2BE6D03F4BBE
:106F00001C6086E7FFF770FF051E00D181E7306047
:106F10004660601CFFF75EFF01002800FFF774FF6A
:106F2000FFF758FF2E000400E1E77B2B5DD1753B96
:106F3000EB60701CFFF74EFF037804007D2BC5D07B
:106F4000FFF752FF061EA86000D162E72000FFF79E
:106F500041FF01003000FFF779FEFFF73BFF0028FB
:106F600000D156E7002433693461336203783A2B49
:106F700002D0224B186062E70130FFF72BFF0100BF
:106F80003000FFF741FFFFF725FF0400002C00D180
:106F90003FE723782C2B02D07D2B97D0AFE7FFF76C
:106FA00023FF051E00D134E730604660601CFFF708
:106FB00011FF01002800FFF749FEFFF70BFF002833
:106FC00000D126E700242B692C612B6203783A2B31
:106FD000CFD10130FFF7FEFE01002800FFF714FFBC
:106FE000FFF7F8FE2E000400D0E7044B1E6010E708
:106FF000F58A0D10FA8A0D10008B0D10D0AD020825
:107000000849094A002803D1084B0B60084B07E0E8
:107010000368002B00D1054B0B604368002BF5D0B3
:107020001360704780A102087CA1020889760D10C8
:107030009D760D10F8B5802604007600002C00D156
:10704000F8BDE3682768334204D1A068002801D066
:10705000FFF7F0FFE3680B4D334204D120690028AD
:1070600001D02B6898478022E3689200134204D134
:10707000206A002801D02B68984720002B68984789
:107080003C00DBE77CA10208F7B505000E00019289
:10709000FFF7AAFE0023134F04003B6098420CD078
:1070A0002800FFF797FE01002000FFF7ADFE051E48
:1070B00005D12000FFF7BEFF00242000FEBD019B8C
:1070C000002B0AD0FFF786FE03780500002B04D0C2
:1070D0002000FFF7AFFF3D60EEE7002EEDD03560FA
:1070E000EBE7C046D0AD0208002210B51100FFF753
:1070F000CBFF10BD0300093B0122042B02D920382D
:107100004242424110007047F0B5002517000600CA
:107110002C0089B003930E9B02901B0CDBB20493EE
:107120000E9B00911B0ADBB205930E9BDBB207930B
:10713000731C069333780193002B08D0009B002B1F
:1071400022DB029A731C9B1A009A9A421CDA0E9B4D
:10715000DBB2002B00D1B4E0019A9A4200D0AEE03D
:10716000009B002B06DB029A731C9B1A009A934229
:1071700000DDA4E0B31C7678032D00D9A1E028003F
:1071800000F0ACF88989637B0198FFF7B3FF002812
:1071900039D1079B019A9342D9D04F4E110030004C
:1071A00000F072FB031E08D1049B019A93420BD09E
:1071B000059B93426FD133003F33032D23D8280022
:1071C00000F08CF80510233533003E33F5E7002F2F
:1071D00006D0039A94425ED23F4A9B1A9B003B55CD
:1071E000012510E0621C002F0BD003998A4252D275
:1071F00039493C195B1A2178181101431B01217090
:10720000BB5414000225069E92E7621C002F0BD08F
:1072100003998A423FD230493C195B1A2178981071
:1072200001439B012170BB5414000325EBE7002FA1
:1072300008D0039A94422ED227493A195B1A117842
:107240000B43137001340025DDE71D00002E22D012
:10725000009B002B22DB029B009AEB1A9A421DDA5C
:10726000019BB34217D1009B002B04DD029B009AC7
:10727000EB1A93420FDC2E786B1C029A9D1A002E9B
:1072800004D0009B002B11DBAB420FDA002F18D08B
:107290003B5D002B15D00124644219E03000FFF75C
:1072A00029FF0028DCD02E780135CFE73000FFF72A
:1072B00021FF0028EFD0029B5E5D0135DFE7002D46
:1072C000E9D1039B9C42E6D2002F01D000233B551D
:1072D000200009B0F0BDC046058B0D1002B4714608
:1072E00049084900095C49008E4402BC7047C04609
:1072F000002243088B4274D303098B425FD3030AF5
:107300008B4244D3030B8B4228D3030C8B420DD307
:10731000FF22090212BA030C8B4202D31212090295
:1073200065D0030B8B4219D300E0090AC30B8B42D3
:1073300001D3CB03C01A5241830B8B4201D38B0381
:10734000C01A5241430B8B4201D34B03C01A524126
:10735000030B8B4201D30B03C01A5241C30A8B4269
:1073600001D3CB02C01A5241830A8B4201D38B0254
:10737000C01A5241430A8B4201D34B02C01A5241F8
:10738000030A8B4201D30B02C01A5241CDD2C3096A
:107390008B4201D3CB01C01A524183098B4201D3E6
:1073A0008B01C01A524143098B4201D34B01C01AD1
:1073B000524103098B4201D30B01C01A5241C30849
:1073C0008B4201D3CB00C01A524183088B4201D3B8
:1073D0008B00C01A524143088B4201D34B00C01AA4
:1073E0005241411A00D20146524110467047FFE710
:1073F00001B5002000F006F802BDC0460029F7D014
:1074000076E770477047C046002B11D1002A0FD194
:10741000002900D1002802D00021C943081C07B46C
:10742000024802A14018029003BDC046D9FFFFFFE9
:1074300003B4684601B5029800F030F8019B9E46FF
:1074400002B00CBC7047C046F0B5CE4647461504A6
:107450002D0C2E0080B50704140C3F0C9946030C2C
:107460007E435D43674363437F19340CE4199C46B4
:10747000A54203D980235B029846C4444B4643434C
:107480005143250C36046544360C2404A4195B19B9
:10749000591820000CBC90469946F0BDF0B54F46F7
:1074A0004646D646C0B5040082B00D0091469846C7
:1074B0008B422FD82CD04146484600F0CFF8290007
:1074C0000600200000F0CAF8331A9C46203B9A467A
:1074D00000D576E04B46524693401F004B4662462D
:1074E00093401E00AF4228D825D05346A41BBD416F
:1074F000002B00DA7BE0002200230092019301239D
:10750000524693400193012362469340009318E052
:107510008242D0D900220023009201930A9B002BC3
:1075200001D01C605D600098019902B01CBC9046BF
:107530009946A246F0BDA342D7D90022002300926B
:1075400001936346002BE9D0FB0798464146720839
:107550000A437B0866460EE0AB4201D1A2420CD83A
:10756000A41A9D41012024196D410021013E2418D7
:107570004D41002E06D0AB42EED9013E24196D419B
:10758000002EF8D100980199534600196941002B4B
:1075900023DB2B005246D3402A006446E2401C0005
:1075A00053461500002B2DDB26005746BE40330006
:1075B00026006746BE403200801A99410090019132
:1075C000ACE7624620239B1A4A46DA406146130024
:1075D00042468A4017001F4380E7624620239B1AD9
:1075E0002A0066469A402300F3401343D4E76246DC
:1075F000202300219B1A0022009101920122DA40EF
:10760000019280E72023624626009B1ADE402F006D
:10761000B0466646B74046463B003343C8E7C046DF
:107620001C2101231B04984201D3000C10391B0AB2
:10763000984201D3000A08391B09984201D3000976
:10764000043902A2105C40187047C04604030202CD
:1076500001010101000000000000000010B5002938
:1076600003D1FFF7DDFF203002E0081CFFF7D8FF51
:1076700010BDC04610B50A22002100F0F7F910BD78
:10768000EC3000687047000010B5034B010018682B
:1076900000F08AF810BDC04684A1020810B5034B63
:1076A0000100186800F036F810BDC04684A1020839
:1076B00082B0002900D101A9101E06D0002B06D0EF
:1076C00013780B601078431E984102B07047022077
:1076D0004042FAE730B50024A24201D1002005E083
:1076E000035D651C0C5DA34201D0181B30BD2C004E
:1076F000F2E7002310B59A4200D110BDCC5CC4540F
:107700000133F8E703001218934200D17047197053
:107710000133F9E770B50500002910D00C1F23686C
:10772000002B00DAE418280000F0C0F91D4A1368A5
:10773000002B05D163601460280000F0B8F970BD1B
:10774000A34209D9216860188342F3D118685B68A5
:1077500041182160EEE713005A68002A01D0A242C6
:10776000F9D919685818A0420BD12068091858187F
:1077700019608242E0D110685268411819605A605D
:10778000DAE7A04202D90C232B60D5E72168601804
:10779000824203D1106852684118216062605C60C7
:1077A000CAE7C046D4AD0208032370B5CD1C9D4383
:1077B000083506000C2D1ED20C25A9421DD830001C
:1077C00000F074F9254A14682100002919D1244CCD
:1077D0002368002B03D1300000F044F8206029001A
:1077E000300000F03FF8431C2BD10C2330003360F5
:1077F00000F05DF903E0002DDFDA0C233360002098
:1078000070BD0B685B1B19D40B2B03D90B60CC1814
:10781000256003E04B688C420DD11360300000F00E
:1078200046F9200007220B30231D9043C31AE7D0EE
:107830005A42E250E4E763600C00EFE70C0049684D
:10784000C3E70323C41C9C43A042E1D0211A3000AB
:1078500000F008F8431CDBD1C7E7C046D4AD0208EE
:10786000D8AD0208002370B5064C0500080023605F
:1078700000F01EF9431C03D12368002B00D02B60BD
:1078800070BDC04604B00208C9B20378002B04D012
:107890008B4200D170470130F7E74B4259414942D2
:1078A0000840F7E702780B78002A03D00130013155
:1078B0009A42F7D0D01A704703000A7801311A7043
:1078C0000133002AF9D17047002330B59A420AD01B
:1078D000013AC45CCD5CAC4204D1934202D0013386
:1078E000002CF6D1631B180030BD30B50500002A0E
:1078F00000D130BD0C78013A6B1C2C700131002C8A
:1079000005D19A189A42F4D01C700133FAE71D0091
:10791000EDE70000F0B51F000E008DB00B90029156
:10792000039212983478FFF7ABFE082200194378CF
:10793000751C134053D12D2C53D17478B51C0133D1
:107940000193002F00D18AE0102F0AD1302C08D1EA
:1079500020222B789343582B00D07AE010276C78A4
:107960000235019B002B41D1013B04933E4B059313
:107970003A00FB17049805990893FFF745FD00238B
:1079800009900E00002000210A922200303A092AB4
:1079900031D81400A7423DDD5A1C1DD0B14236D863
:1079A00002D1099B984232D8099B834206D18E426C
:1079B00004D101230A9A5B42A2420DDB0B000200B4
:1079C00008993800FFF740FDE31706940793069BDC
:1079D000079CC018614101232C780135D5E72E00A2
:1079E0009FE72B2CACD1B51C7478A9E70023049336
:1079F00080231B06BBE72200413A192A01D8373CF5
:107A0000C8E72200613A192A04D8573CC2E701238B
:107A10005B42E1E75A1C09D10B9A23331360039BA5
:107A200004980599002B0ED10DB0F0BD019A002AE3
:107A300004D006000F0000217042B941039A002AC9
:107A4000F2D0002B01D06B1E0293039B029A1A60A6
:107A5000EAE73024002F00D083E7082781E7302CA5
:107A600000D175E70A277CE7FFFFFF7F37B51300DA
:107A7000064A05001068046A002C00D1044C0A0074
:107A800000942900FFF746FF03B030BD84A102082F
:107A9000E8A102080B1E04D0FF2A04D98A23036040
:107AA0008B3B180070470A700123FAE77047704754
:107AB000044A1368002B00D1034B181810601800FB
:107AC0007047C046DCAD020800000208F8B5C046A9
:107AD000F8BC08BC9E467047F8B5C046F8BC08BC68
:107AE0009E4670470000000001B40248844601BC75
:107AF000604700BF1DA5020801B40248844601BCCE
:107B0000604700BF01A7020801B40248844601BCD7
:107B1000604700BFEFA3020801B40248844601BCDD
:107B2000604700BF03A70208000000000700010330
:107B300000000100030300003F00010300000F00EC
:107B4000C0102040030300004000010300000F00AC
:107B500000112040030300003F00010300000F005C
:107B600040112040030300007F00010300000F00CC
:107B700080112040000300000F00010300000F00EF
:107B800040122040030300003F00010300000F00EB
:107B900080122040000300000F00010300000F00CE
:107BA00000162040000300000F00010300000F003A
:107BB00040162040000300000F00010300000F00EA
:107BC00080162040000300000F00010300000F009A
:107BD00000172040000300007F00010300000F0099
:107BE00040002040030300007F00010300000F005D
:107BF000C0002040030300007F00010300000F00CD
:107C000000012040030300007F00010300000F007B
:107C100080012040000001400900000300000F0027
:107C2000010300000F00000000410140130007079E
:107C300000007F00802224400103010000000707AC
:107C40000000030000212440010301000100070798
:107C500000000300C02024400103010002000707C8
:107C600000000F00802024400103010005000505ED
:107C700000017E00402024400103010006000303B0
:107C800000017E0000202440010301000CC0000719
:107C900000000F0000222440010301000D0001013B
:107CA0000001700040222440010301000E00030384
:107CB00000000100C0212440010301000FC007079C
:107CC00000000F0080212440010301001000030385
:107CD0000000040040212440010301000CDF0007E4
:107CE00000000F00402224400103010070726F76F3
:107CF0005F726571007265736F75726365730042C0
:107D00004F4F5400555047524144450073697A65BE
:107D1000006C61756E6368006D6F6E6F746F6E6975
:107D20006300656E637279707400656E637279705A
:107D3000745F6B65795F6964006261636B75700085
:107D4000626F6F745F6175746800757067726164EB
:107D5000655F6175746800736D69665F6964007260
:107D60006570726F6772616D007374617274007216
:107D70006570726F766973696F6E00626F6F745FA2
:107D80006C6F61646572006B6579735F616E645FCF
:107D9000706F6C6963696573006D30700070657237
:107DA0006D697373696F6E00636F6E74726F6C00D0
:107DB0006B6579006D340073797374656D00737948
:107DC0007363616C6C006D6D696F00726D6100644E
:107DD000657374726F795F6675736573006465733C
:107DE00074726F795F666C61736800707265736539
:107DF0006E74006669726D77617265006365727496
:107E000069666963617465006F70656E00646973AB
:107E100061626C656400656E61626C656400616CD2
:107E20006C6F77656400646562756700776F756E67
:107E300064696E6700626F6F745F7570677261640A
:107E400065007479706500617272617900697465AA
:107E50006D73006E756D62657200696E746567653D
:107E60007200626F6F6C65616E00737472696E6729
:107E7000006D6178696D756D006D696E696D756D08
:107E8000007065726970686572616C73006261731D
:107E9000655F61646472657373006D656D6F7269AF
:107EA000657300776F726B666C6173680073666CE4
:107EB000617368007372616D00736F6674776172CD
:107EC00065006361706162696C69747900464C4158
:107ED00053485F5043315F53504D00464C41534827
:107EE0005F50433200464C4153485F504333004695
:107EF0004C4153485F50433400464C4153485F4D1A
:107F000041494E5F434F444500464C4153485F4D05
:107F100041494E5F584F00464C4153485F4D4149DF
:107F20004E5F4441544100464C4153485F535550C5
:107F300045525649534F525900464C4153485F579A
:107F40004F524B5F53454355524500464C415348B1
:107F50005F574F524B005352414D5F5043305F507B
:107F6000524956005352414D5F5043305F50554285
:107F7000005352414D5F53504D5F5052495600538C
:107F800052414D5F53504D5F505542005352414D49
:107F90005F5043315F50524956005352414D5F503C
:107FA00043325F50524956005352414D5F50433364
:107FB0005F50524956005352414D5F5043345F5019
:107FC000524956005352414D5F4D41494E00535264
:107FD000414D5F44415000534D49465F434F444536
:107FE00000534D49465F584F00534D49465F444149
:107FF00054410000000021400000254000000140E5
:1080000000003440000024400000314000003240B5
:1080100000001F4100002340000011400101010148
:108020000101010101101010800019005500F0003D
:108030000501053B04101C01010000000FC00000F9
:108040000004000001010101011D3A577896000863
:108050002000101208000000001F00000010000F98
:10806000002000023F06080E00080009000A000B6D
:1080700024282C3034000000100000009000000084
:1080800088000000080000008000000004F00000EC
:1080900000F00000400200002005A000D001000117
:1080A0008001A0012000000010000000433A5C475E
:1080B00069744C61622D52756E6E65725C62756991
:1080C0006C64735C32643334316331325C305C72C3
:1080D00065706F5C6379626F6F746C6F61646572F9
:1080E0005C70736F633670646C5C64726976657221
:1080F000735C696E636C7564652F63795F69706327
:108100005F6472762E6800433A2F4769744C61624F
:108110002D52756E6E65722F6275696C64732F32A5
:10812000643334316331322F302F7265706F2F63B7
:1081300079626F6F746C6F616465722F70736F63B7
:108140003670646C2F647269766572732F736F7505
:108150007263652F63795F6770696F2E6300433ABE
:108160005C4769744C61622D52756E6E65725C621B
:1081700075696C64735C32643334316331325C3002
:108180005C7265706F5C6379626F6F746C6F616451
:1081900065725C70736F633670646C5C6472697670
:1081A0006572735C696E636C7564652F63795F6774
:1081B00070696F2E6800433A2F4769744C61622DD5
:1081C00052756E6E65722F6275696C64732F3264BE
:1081D0003334316331322F302F7265706F2F6379F2
:1081E000626F6F746C6F616465722F70736F63364A
:1081F00070646C2F647269766572732F736F757219
:1082000063652F63795F6970635F6472762E6300C4
:10821000433A2F4769744C61622D52756E6E6572D8
:108220002F6275696C64732F326433343163313279
:108230002F302F7265706F2F6379626F6F746C6F60
:10824000616465722F70736F633670646C2F647233
:1082500069766572732F736F757263652F63795FCB
:108260006970635F706970652E6300433A2F4769D8
:10827000744C61622D52756E6E65722F6275696CF9
:1082800064732F32643334316331322F302F72658F
:10829000706F2F6379626F6F746C6F616465722F9A
:1082A00070736F633670646C2F6472697665727375
:1082B0002F736F757263652F63795F70726F742EA1
:1082C0006300433A2F4769744C61622D52756E6E9C
:1082D00065722F6275696C64732F32643334316355
:1082E00031322F302F7265706F2F6379626F6F7428
:1082F0006C6F616465722F70736F633670646C2F7E
:10830000647269766572732F736F757263652F631C
:10831000795F736D69662E630000010010008000B4
:10832000E80310000001A00F00FA433A2F476974D8
:108330004C61622D52756E6E65722F6275696C6448
:10834000732F32643334316331322F302F726570C2
:108350006F2F6379626F6F746C6F616465722F70D9
:10836000736F633670646C2F647269766572732FF5
:10837000736F757263652F63795F736D69665F6D87
:10838000656D736C6F742E6300433A2F4769744CAC
:1083900061622D52756E6E65722F6275696C6473C1
:1083A0002F32643334316331322F302F7265706F66
:1083B0002F6379626F6F746C6F616465722F707375
:1083C0006F633670646C2F647269766572732F7395
:1083D0006F757263652F63795F737973636C6B2E4E
:1083E0006300433A2F4769744C61622D52756E6E7B
:1083F00065722F6275696C64732F32643334316334
:1084000031322F302F7265706F2F6379626F6F7406
:108410006C6F616465722F70736F633670646C2F5C
:10842000647269766572732F736F757263652F63FB
:10843000795F737973696E742E6300433A2F4769CD
:10844000744C61622D52756E6E65722F6275696C27
:1084500064732F32643334316331322F302F7265BD
:10846000706F2F6379626F6F746C6F616465722FC8
:1084700070736F633670646C2F64726976657273A3
:108480002F736F757263652F63795F737973706D86
:108490002E6300433A2F4769744C61622D52756E0A
:1084A0006E65722F6275696C64732F326433343178
:1084B0006331322F302F7265706F2F6379626F6F67
:1084C000746C6F616465722F70736F633670646C67
:1084D0002F646576696365732F70736F63362F73CE
:1084E0007461727475702F73797374656D5F7073D6
:1084F0006F63365F636D30706C75732E63000000C0
:108500000300000001000000010000000000000066
:1085100005036000040000000100000000000000EE
:108520000100000006046000080000001CC00208F2
:10853000994E0D1050534F43365F464C41534800FF
:1085400034850D10695E0D100000000040850D108F
:10855000B48A0D10000000000000000007000000B9
:108560000100000000000000010000000E000000FB
:1085700011000000000000000000000000000000EA
:1085800000000000000000000000000000000000EB
:1085900000000000000000000000000001000000DA
:1085A0000E000000110000000000000000000000AC
:1085B00000000000000000000000000000000000BB
:1085C00000000000000000000000000000000000AB
:1085D000010000000E00000011000000000000007B
:1085E000000000000000000000000000000000008B
:1085F000000000000000000000000000000000007B
:1086000000000000010000000E000000110000004A
:10861000000000000000000000000000000000005A
:10862000000000000000000000000000000000004A
:108630000000000000000000010000000600000033
:108640001100000000000000000000000000000019
:10865000000000000000000000000000000000001A
:108660000000000000000000000000000100000009
:1086700006000000110000000000000000000000E3
:1086800000000000000000000000000000000000EA
:1086900000000000000000000000000000000000DA
:1086A00001000000000000000000000000000000C9
:1086B00000000000000000000000000000000000BA
:1086C00000000000000000000000000000000000AA
:1086D0000000000001000000000000000000000099
:1086E000000000000000000000000000000000008A
:1086F000000000000000000000000000000000007A
:108700000000000000000000010000000600000062
:108710001D0000000000000000000000000000003C
:108720000000000000000000000000000000000049
:108730000000000000000000000000000100000038
:108740000A0000001D000000000000000000000002
:108750000000000000000000000000000000000019
:108760000000000000000000000000000000000009
:10877000010000000B0000001D00000000000000D0
:1087800000000000000000000000000000000000E9
:1087900000000000000000000000000000000000D9
:1087A00000000000433A5C4769744C61622D5275C9
:1087B0006E6E65725C6275696C64735C32643334CE
:1087C000316331325C305C7265706F5C6379626F0B
:1087D0006F746C6F616465725C70736F6336706424
:1087E0006C5C647269766572735C696E636C7564E7
:1087F000652F63795F737973636C6B2E680000007B
:10880000F4010000140004010A0009050800030037
:1088100063010000020000000300000000000000EF
:10882000000000180000800000000000FC890D100E
:108830006000000000000000FFFFFFFF00000000DC
:108840000000000000000000200000000000000008
:10885000FFFFFFFF0000000000000000000000001C
:108860000200000000000000FFFFFFFF000000000A
:108870000000000000000000EB000000000200000B
:1088800001000000020000000800000002000000DB
:108890003500000000000000FFFFFFFF00000000A7
:1088A00000000000000000000500000000000000C3
:1088B000FFFFFFFF000000000000000000000000BC
:1088C0000400000000000000FFFFFFFF00000000A8
:1088D0000000000000000000060000000000000092
:1088E000FFFFFFFF0000000000000000000000008C
:1088F0000100000000000000FFFFFFFF000000007B
:108900000000000000000000010000000300000063
:10891000000000000000001800000001000000003E
:10892000488A0D106000000000000000FFFFFFFFFC
:108930000000000000000000000000002000000017
:1089400000000000FFFFFFFF00000000000000002B
:10895000000000003800000000020000FFFFFFFFE1
:10896000020000000000000002000000EB00000018
:1089700000020000010000000200000004000000EE
:10898000020000003500000000000000FFFFFFFFB4
:1089900000000000000000000000000005000000D2
:1089A00000000000FFFFFFFF0000000000000000CB
:1089B000000000000400000000000000FFFFFFFFB7
:1089C00000000000000000000000000006000000A1
:1089D00000000000FFFFFFFF00000000000000009B
:1089E000000000000100000000000000FFFFFFFF8A
:1089F0000000000000000000000000000300000074
:108A00000000800078880D10D8880D10C0880D10E7
:108A100048880D100010000030880D1060880D107F
:108A200000010000A8880D1090880D10F0880D102E
:108A300000000000010000000200000041000000F2
:108A4000D8D60000C20100000300000000000001B1
:108A50006C890D10CC890D10B4890D103C890D1056
:108A60000010000024890D1054890D100001000031
:108A70009C890D1084890D10E4890D100000000000
:108A800001000000020000008C000000409C00007B
:108A9000FA000000010000005CA8020801000000CC
:108AA0001400000007008E00010000000000080014
:108AB00000020000A55D0D10D15E0D10E55E0D10E9
:108AC000A15D0D10915D0D100400000077C295F3BB
:108AD00060D2EF7F3552500F2CB67980000100FF35
:108AE00000020001000100030103FF000104000077
:108AF000C0E0F0F8FC6E756C6C0066616C7365002C
:108B000074727565004142434445464748494A4BA3
:108B10004C4D4E4F505152535455565758595A6117
:108B200062636465666768696A6B6C6D6E6F7071AD
:108B300072737475767778797A30313233343536AA
:108B4000373839004300504F534958002E00002059
:108B500020202020202020202828282828202020ED
:108B6000202020202020202020202020202020889D
:108B70001010101010101010101010101010100401
:108B80000404040404040404041010101010101051
:108B90004141414141410101010101010101010145
:108BA000010101010101010101011010101010105B
:108BB0004242424242420202020202020202020215
:108BC0000202020202020202020210101010200031
:108BD0000000000000000000000000000000000095
:108BE0000000000000000000000000000000000085
:108BF0000000000000000000000000000000000075
:108C00000000000000000000000000000000000064
:108C10000000000000000000000000000000000054
:108C20000000000000000000000000000000000044
:108C30000000000000000000000000000000000034
:108C40000000000000000000000000000000000024
:048C50000000000020
:088C540048E8FF7F0100000069
:108C5C0000000D1000A00208C0000000848C0D1054
:088C6C00C0A00208F0060000A0
:108C7400ECA702081C08000000C002089C010000C8
:108C8400CD7E0D10DB7E0D10E57E0D10EF7E0D10F8
:108C9400F97E0D10097F0D10177F0D10277F0D1021
:108CA400397F0D104B7F0D10567F0D10647F0D1012
:108CB400717F0D107F7F0D108C7F0D109A7F0D102A
:108CC400A87F0D10B67F0D10C47F0D10CE7F0D1040
:108CD400D77F0D10E17F0D10E97F0D1000093D00D5
:108CE40000127A0000093D000000D00700093D0091
:108CF400A00F00000400000008890D1014880D1056
:108D0400EFBE0DD0016F0000000000000000020063
:108D140000000000EFBE0DD0026F0000000005004F
:108D24000000020000000000EFBE0DD0036F000041
:108D340000000F0000100000000000009D760D10E0
:108D440089760D1088A102080000000000000000D0
:108D5400000000000000000000000000000000000F
:108D640000000000000000000000000000000000FF
:108D740000000000000000000000000000000000EF
:108D840000000000000000000000000000000000DF
:108D940000000000000000000000000000000000CF
:108DA400000000000000000043000000000000007C
:108DB40000000000000000000000000000000000AF
:108DC400000000000000000043000000000000005C
:108DD400000000000000000000000000000000008F
:108DE400000000000000000043000000000000003C
:108DF400000000000000000000000000000000006F
:108E0400000000000000000043000000000000001B
:108E1400000000000000000000000000000000004E
:108E240000000000000000004300000000000000FB
:108E3400000000000000000000000000000000002E
:108E440000000000000000004300000000000000DB
:108E5400000000000000000000000000000000000E
:108E640000000000000000004300000000000000BB
:108E740000000000000000000000000000000000EE
:108E84000000000000000000957A0D10B1760D106E
:108E9400000000004E8B0D104C8B0D104D8B0D10EF
:108EA4004D8B0D104D8B0D104D8B0D104D8B0D10EA
:108EB4004D8B0D104D8B0D104D8B0D104D8B0D10DA
:108EC400FFFFFFFFFFFFFFFFFFFFFFFFFFFF0000AC
:108ED4000100415343494900000000000000000024
:108EE400000000000000000000000000000000007E
:108EF4000000415343494900000000000000000005
:108F0400000000000000000000000000000000005D
:108F140000000000E9000D10C1000D1080B230B552
:108F2400C00020D0104B07221C682300B0331B88DC
:108F34005A43236AD31819680029FCDA3E210B4BE3
:108F4400062519600A4B0B491960A3210A4BC90075
:108F54005D500A4958505858206A12180020506031
:108F64005A58002AFCDA30BDE0AD0208040126405C
:108F7400080126401E1F0000000026401C050000BA
:108F840010B54378FF2B11D100F0BAF90400032087
:108F940000F0A6F9C3685A680123116819431160E7
:108FA40011681942FCD1200000F092F910BDF7B508
:108FB40000900020019100F093F93F4D06002B68CA
:108FC4001A005033B43214681B780419002B5AD099
:108FD40000F0B6F9070003281BD000F091F9374AD6
:108FE400374B0500D358002B3EDA364A01213000B6
:108FF40000F0B6F9002837D10198FFF78FFF009BE6
:10900400002B3ED02368002BFCDB00F081F9040028
:109014002BE0062000F064F92B68B4331B68C018F9
:109024000368002B02DA284C2000FEBD002000F06B
:109034005FF9264B9842F6D00023254A190012689E
:10904400012000F085F90025A842ECD1002000F0B1
:109054004FF91E4A1F4B904203D09D42E3D0013585
:10906400F4E79D42B9D1DEE7174C032F05D1012166
:10907400002000F05DF90028F9D1280000F028F95B
:10908400D2E7154CF1E700F03BF90E4A0500012147
:10909400300000F065F9002809D1009B002B08D0AE
:1090A4002368002BFCDB00F033F90400E5E7064CF1
:1090B400E3E7094CE1E7C046E0AD020800002640C2
:1090C4001C05000008A802080500520001018800E0
:1090D40018A80208F049020001005000F7B56E4DCF
:1090E40004002A68536800931300B03319880723D7
:1090F4004B43126A9B181A68002AFCDA00F010F934
:109104002A681300B033198807234B43212800D061
:1091140096E0116A5B180221D8680143D960D968C6
:10912400C9072FD508208446944460461600D968A0
:10913400C06F0191116888360818356807684919A5
:109144000D683902FF273F040F40694689882D0ABC
:109154002D0639432943D960902103684F4D0901F5
:109164002B400B430360136830681B1818680540D4
:109174002943196013686246D26F9A1812683268DC
:109184009B181B68444D2A681300B03319880723C1
:109194004B43126A9B1800225A600423404A116907
:1091A4000B431361012C50D030BF2A681300B03335
:1091B400198807234B43126A9B181A68002AFCDAA1
:1091C40000F0AEF8212842D1296807220B000124BF
:1091D400B0331B8800205A430B6AD318DD6825423C
:1091E4001CD0080008300D68C06F2C4E2818056884
:1091F400DB6835401B0C1B061B0C2B4303600B0068
:10920400883318680B6818180B6A0568D318DB686C
:109214002E401B0E1B023343036020000B6A022105
:10922400D218D3688B43D3601B4B1A681300B03336
:10923400198807234B43126A9B1800225A60FEBD0B
:10924400126A9B18174ADA609CE720BFADE700203A
:10925400009BFC331B698342E6D1A320124B1349C4
:10926400134A144FC0000E681D5814680F60062777
:109274001F503E20106010483E371F501F58002FCB
:10928400FCDA00980D4FFC3007610E60A321C90081
:109294005D5001201460C7E7E0AD0208FF00FFFF46
:1092A40000ED00E024A80208000026400801264042
:1092B400040126401E1F00001C050000AAAAAAAA39
:1092C400FEE7024A1368002BFCDB704700012640CE
:1092D40001B40248844601BC604700BF1B1D0D1049
:1092E40001B40248844601BC604700BF0D1E0D1046
:1092F40001B40248844601BC604700BF21280D1018
:1093040001B40248844601BC604700BF131D0D1020
:1093140001B40248844601BC604700BF411E0D10E1
:1093240001B40248844601BC604700BF81440D106B
:1093340001B40248844601BC604700BFAD270D104C
:1093440001B40248844601BC604700BFCD4D0D10F6
:1093540001B40248844601BC604700BF29250D10B2
:1093640001B40248844601BC604700BF31230D109C
:10FE0000FC010000211221010000000000000000A0
:10FE100000000D1000FE0000000001007D00000049
:10FE20000100000000DA0F100000000000000000D8
:10FE300000000000000000000000000000000000C2
:10FE400000000000000000000000000000000000B2
:10FE500000000000000000000000000000000000A2
:10FE60000000000000000000000000000000000092
:10FE70000000000000000000000000000000000082
:10FE80000000000000000000000000000000000072
:10FE90000000000000000000000000000000000062
:10FEA0000000000000000000000000000000000052
:10FEB0000000000000000000000000000000000042
:10FEC0000000000000000000000000000000000032
:10FED0000000000000000000000000000000000022
:10FEE0000000000000000000000000000000000012
:10FEF0000000000000000000000000000000000002
:10FF000000000000000000000000000000000000F1
:10FF100000000000000000000000000000000000E1
:10FF200000000000000000000000000000000000D1
:10FF300000000000000000000000000000000000C1
:10FF400000000000000000000000000000000000B1
:10FF500000000000000000000000000000000000A1
:10FF60000000000000000000000000000000000091
:10FF70000000000000000000000000000000000081
:10FF80000000000000000000000000000000000071
:10FF90000000000000000000000000000000000061
:10FFA0000000000000000000000000000000000051
:10FFB0000000000000000000000000000000000041
:10FFC0000000000000000000000000000000000031
:10FFD0000000000000000000000000000000000021
:10FFE0000000000000000000000000000000000011
:10FFF000000000000000000000000000000028D306
:04000005100D4B335C
:00000001FF
